S024000062696E2F6F70656E62746C5F6F6C696D65785F73746D3332653430372E737265639F
S3150800000064360020419400082D9400082D940008B9
S315080000102D9400082D9400082D9400082D940008AE
S315080000202D9400082D9400082D9400082D9400089E
S315080000302D9400082D9400082D9400082D9400088E
S315080000402D9400082D9400082D9400082D9400087E
S315080000502D9400082D9400082D9400082D9400086E
S315080000602D9400082D9400082D9400082D9400085E
S315080000702D9400082D9400082D9400082D9400084E
S315080000802D9400082D9400082D9400082D9400083E
S315080000902D9400082D9400082D9400082D9400082E
S315080000A02D9400082D9400082D9400082D9400081E
S315080000B02D9400082D9400082D9400082D9400080E
S315080000C02D9400082D9400082D9400082D940008FE
S315080000D02D9400082D9400082D9400082D940008EE
S315080000E02D9400082D9400082D9400082D940008DE
S315080000F02D9400082D9400082D9400082D940008CE
S315080001002D9400082D9400082D9400082D940008BD
S315080001102D9400082D9400082D9400082D940008AD
S315080001202D9400082D9400082D9400082D9400089D
S315080001302D9400082D9400082D9400082D9400088D
S315080001402D9400082D9400082D9400082D9400087D
S315080001502D9400082D9400082D9400082D9400086D
S315080001602D9400082D9400082D9400082D9400085D
S315080001702D9400082D9400082D9400082D9400084D
S315080001802D9400082D940008704700BF704700BFE3
S31508000190704700BF08B50020C4F20200012103F031
S315080001A053FD10F1FF3018BF012008BD00B589B016
S315080001B000230093019302930393049305930693F4
S315080001C0079349F2E850C0F60000694605F072FE4A
S315080001D048B9009B002043B19DF8080080F0100044
S315080001E0C0F3001001E00020FFE709B05DF804FB4A
S315080001F049F2E850C0F60000704700BF08B540F263
S315080002000010C2F20000002380F8243249F2086187
S31508000210C0F600010A2205F0ABFA30B940F2001325
S31508000220C2F20003012283F8242208BD38B540F241
S315080002300013C2F2000393F82432012B05D140F2D1
S315080002400010C2F2000005F05FFD4FF4A054C4F29E
S31508000250010440252046294603F016FF0028F9D058
S3150800026049F2E850C0F6000005F04AFE38BD00BF66
S3150800027008B540F20013C2F2000393F82432012BAA
S3150800028005D140F20010C2F2000005F03DFD08BDA0
S3150800029070B5064640F20013C2F2000393F8243202
S315080002A0012B10D140F20011C2F2000105F0C8FE80
S315080002B0002808DA40F20010C2F20000002380F895
S315080002C0243205F021FD317889B14FF4A054C4F2E7
S315080002D001048025204603F0CFFE2046294603F078
S315080002E0D3FE0028F9D016F8011F0029F2D170BDF7
S315080002F080B582B003F0CEFE0120014603F02CFD46
S315080003000124009400278DF804708DF807700225E3
S315080003108DF805503846C4F20200694603F04CFCD5
S315080003202020214603F04EFD0420214603F014FD4B
S315080003304FF40066C4F2020630460621082203F08E
S3150800034089FC30460721082203F084FC8DF80670E4
S315080003508DF807408DF80450402300938DF805501A
S315080003603046694603F028FC8DF804508023009334
S315080003703046694603F020FC2846214603F0ECFC8B
S315080003804FF48066C4F2020630460521092203F0BE
S3150800039061FC30460621092203F05CFC60230093C9
S315080003A08DF804508DF805508DF806708DF80740C5
S315080003B03046694603F000FC4FF0C060214603F062
S315080003C0EFFC07F063F907F06FF9FCE720230B80D1
S315080003D040F20000C2F20000704700BF08B590F86E
S315080003E01231032B01D108F041FF002008BD00BFE0
S315080003F008B508F03BFF002008BD00BF08B5084651
S3150800040008F08CFF002008BD08B50B7813F0600FC4
S3150800041028D14B780A2B12D00B2B18D0062B21D1BA
S315080004204B881B0A212B05D1CA88172A28BF1722F1
S315080004300D4901E00D49172200F080FA12E040F25A
S315080004402831C2F20001012200F078FA0AE08B781E
S3150800045033B940F22833C2F2000300221A6001E0E1
S3150800046000F0D4FA002008BD120000200900002080
S3150800047010B50446812101F02BFA2046012101F02E
S3150800048027FA002010BD00BF10B50446812140227E
S31508000490022301F0F3F9204601214022022301F04C
S315080004A0EDF92046012141F6E802C2F20002402396
S315080004B001F028FA002010BD41F6E800C2F200005B
S315080004C0704700BF12230B8040F26C00C2F2000096
S315080004D0704700BF04230B8040F26800C2F2000098
S315080004E0704700BF10B50A4641F62C14C2F2000444
S315080004F049F21860C0F60000214600F0F7FC2046D5
S3150800050010BD00BF10B50A4641F62C14C2F200040D
S3150800051049F22C60C0F60000214600F0E7FC2046B0
S3150800052010BD00BF10B50A4641F62C14C2F20004ED
S3150800053049F23C60C0F60000214600F0D7FC204690
S3150800054010BD00BF10B50A4641F62C14C2F20004CD
S3150800055049F24C60C0F60000214600F0C7FC204670
S3150800056010BD00BF10B50A4641F62C14C2F20004AD
S3150800057049F25460C0F60000214600F0B7FC204658
S3150800058010BD00BF704700BF704700BF704700BF6F
S3150800059008B5FFF7FBFD08BD08B5FFF7F9FD08BD6F
S315080005A008B50120FFF7F0FD08BD00BF08B500201B
S315080005B0FFF7EAFD08BD00BFF0B583B0012001468C
S315080005C003F0CAFB4FF4C853009303278DF8057050
S315080005D002238DF8043000268DF806608DF8076032
S315080005E03446C4F202042046694603F0E5FA20467A
S315080005F008210A2203F02EFB20460B210A2203F0CB
S3150800060029FB20460C210A2203F024FB4FF4007331
S3150800061000938DF805708DF8046001258DF8065055
S315080006208DF807602046694603F0C6FA4FF48063E2
S3150800063000938DF806508DF807508DF80570204602
S31508000640694603F0B9FA20460A210A4603F002FB76
S315080006504FF48040294603F0B5FB8020294603F075
S315080006608DFB03B0F0BD00BF704700BF1C2202E03F
S3150800067000BF013BFCD10138B0F1FF3F01D0134662
S31508000680F6E7704708B54FF47A7303FB00F0FFF7F7
S31508000690EDFF08BD10B50446D0F8E8351B69984744
S315080006A0032384F81231002010BD00BF08B590F866
S315080006B0123180F81331042380F81231D0F8E83566
S315080006C0DB689847002008BD08B5D0F8E435DB6933
S315080006D003B19847002008BD08B5D0F8E4351B6A71
S315080006E09847002008BD00BF08B5D0F8E4355B6A16
S315080006F09847002008BD00BF10B50446D0F8E83575
S315080007005B699847012384F81531002010BD00BFA6
S3150800071010B50446D0F8E8359B699847D4F8E4350F
S315080007205B68204600219847002084F8150110BD13
S3150800073010B50446002140220B4601F09FF82046DA
S3150800074080214022002301F099F8012384F8123110
S31508000750D4F8E8355B68A0789847002010BD00BF3C
S3150800076010B582B00446694600F02EF99DF80010CF
S3150800077001F01F03012B08D013B1022B0AD00EE09B
S315080007802046694600F050F90EE02046694600F01A
S31508000790F5FA09E02046694600F00CFB04E020461D
S315080007A001F0800101F0E4F8002002B010BD00BF9E
S315080007B010B504460A4600294AD190F81131022B91
S315080007C037D1D0F83821D0F824319A4210D9D21A24
S315080007D0C0F83821C178012902BFD0F828115B1862
S315080007E0C0F82831D4F8281192B200F0B9F820E000
S315080007F0D0F83C21B2FBF3F103FB112161B9934216
S315080008000AD8D0F840319A4206D20A4600F0A8F82B
S315080008100023C4F840310CE0D4F8E435DB682BB18A
S3150800082094F81221032A01D120469847204600F061
S31508000830BBF894F81631012B14D1226941F6281316
S31508000840C2F200031B685360002384F8163109E0DE
S31508000850D0F8E4355B692BB190F81211032901D160
S3150800086011469847002010BD10B504460A4651BBEC
S3150800087090F81131032B30D1D0F89023D0F87C337F
S315080008809A4213D9D21AC0F89023C178012902BF17
S31508000890D0F88013C918C0F880139A4228BF1A46A0
S315080008A0D4F8801392B200F065F816E0D0F8E43573
S315080008B01B6923B190F81221032A00D198472046D4
S315080008C000F062F809E0D0F8E4359B692BB190F89E
S315080008D01211032901D111469847002010BD00BF07
S315080008E0F8B504460D4616461F46FFF765FEC4F8DA
S315080008F0E475069BC4F8E835C4F8EC652046294635
S3150800090000F06EFFD4F8E8351B6898472046FFF7D5
S31508000910ABFEF8BD10B50446D0F8E4351B68984719
S31508000920D4F8E8359B689847002010BD08B5D0F87C
S31508000930E4355B689847002008BD00BF38B5044613
S315080009400D461346C4F83C21C4F83821022280F823
S31508000950112100212A4600F0F1FF002038BD00BF12
S3150800096010B50C4613460021224600F0E7FF00208A
S3150800097010BD00BF10B50C4613460021224600F0F4
S31508000980C1FF002010BD00BF10B50446042380F83F
S31508000990113100210A460B4600F0D0FF204600F030
S315080009A0FDFE002010BD00BF10B50446052380F8E3
S315080009B0113100210A460B4600F0A4FF204600F03C
S315080009C0EDFE002010BD00BF90F8CC350B7090F8F6
S315080009D0CD354B7090F8CF2590F8CE3503EB022332
S315080009E04B8090F8D12590F8D03503EB02238B8005
S315080009F090F8D32590F8D23503EB02239BB2CB802F
S31508000A00C0F84031012380F81131704710B504460B
S31508000A10802100F0ADFF2046002100F0A9FF204606
S31508000A2000F0BCFE10BD00BF70B582B005460C468E
S31508000A304B78092B00F29C81DFE813F02301820131
S31508000A409A0144019A0193000A009A010301B80029
S31508000A506288130A013B062B6DD8DFE803F00415FC
S31508000A60226C6C646800D0F8EC351B6880780DF150
S31508000A70060198470146E388402B03D095F81231C2
S31508000A80012B5CD108235FE0D0F8E4359B6A8078B7
S31508000A900DF106019847014602234370C5F8F00593
S31508000AA04DE0D2B2052A3AD8DFE802F0030C151E4B
S31508000AB02730D0F8EC355B6880780DF10601984749
S31508000AC001463CE0D0F8EC359B6880780DF10601CC
S31508000AD09847014633E0D0F8EC35DB6880780DF1AD
S31508000AE00601984701462AE0D0F8EC351B6980785C
S31508000AF00DF106019847014621E0D0F8EC355B690F
S31508000B0080780DF106019847014618E0D0F8EC35D3
S31508000B109B6980780DF10601984701460FE021464A
S31508000B20FFF774FF27E12146FFF770FF23E121460F
S31508000B30FFF76CFF1FE12146FFF768FF1BE1BDF8D1
S31508000B400630002B00F01781E288002A00F0138196
S31508000B50934238BF1A46ADF806202846FFF7EEFE40
S31508000B6009E1A388EBB9E388DBB9A67806F07F0626
S31508000B7090F81231032B03D12146FFF747FFFAE01D
S31508000B8080F81461314600F033FF2846FFF7FCFE73
S31508000B901EB1022385F81231EDE0012385F81231E2
S31508000BA0E9E028462146FFF731FFE4E0A27840F263
S31508000BB03833C2F200031A70012A03D92146FFF717
S31508000BC025FFD8E090F81231022B02D0032B10D063
S31508000BD033E05AB180F81021032380F81231114608
S31508000BE0FFF798FE2846FFF7CFFEC4E0FFF7CCFED6
S31508000BF0C1E05AB9022380F81231002180F8101199
S31508000C00FFF794FE2846FFF7BFFEB4E090F81011F0
S31508000C108A420FD0FFF78AFE40F23833C2F2000349
S31508000C20197885F810112846FFF774FE2846FFF74D
S31508000C30ABFEA0E0FFF7A8FE9DE02146FFF7E6FE23
S31508000C4099E0E388012B03D02146FFF7DFFE92E007
S31508000C5090F81231022B02D0032B08D00DE040F297
S31508000C603431C2F200010122FFF768FE83E005F580
S31508000C7088710122FFF762FE7DE02146FFF7C6FE76
S31508000C8079E090F81231023B012B17D840F22C3349
S31508000C90C2F2000301221A60D0F818312BB140F2D3
S31508000CA02C33C2F2000303221A60284640F22C3184
S31508000CB0C2F200010222FFF741FE5CE02146FFF77F
S31508000CC0A5FE58E06388012B0AD1C0F81831D0F880
S31508000CD0E4359B68214698472846FFF755FE4AE0C3
S31508000CE0022B48D1A38813F0FF0F44D1026952683A
S31508000CF01B0A013B042B17D8DFE803F003070B0F89
S31508000D001300012363F306120EE0022363F30612AF
S31508000D100AE0032363F3061206E0042363F30612CC
S31508000D2002E0052363F3061241F62813C2F2000314
S31508000D301A60012385F816312846FFF725FE1AE0C2
S31508000D4090F81231023B012B0ED86388012B12D181
S31508000D500023C0F81831D0F8E4359B682146984737
S31508000D602846FFF711FE06E02146FFF74FFE02E090
S31508000D702146FFF74BFE002002B070BD38B5044689
S31508000D800D4690F81231032B0FD10B79012B09D898
S31508000D90D0F8E4359B689847EB8843B92046FFF7B7
S31508000DA0F3FD04E0FFF732FE01E0FFF72FFE002017
S31508000DB038BD00BF38B505460C468A88D1B2637877
S31508000DC0012B27D0002B48D0032B40F08D8090F8BC
S31508000DD01231022B02D0032B07D017E011F07F0F38
S31508000DE000F0828000F0C4FD7EE0638823B911F02C
S31508000DF07F0F01D000F0BCFDD5F8E4359B68284686
S31508000E00214698472846FFF7BFFD6DE02146FFF7C4
S31508000E10FDFD69E090F81231022B02D0032B06D0B3
S31508000E2017E011F07F0F5FD000F0A2FD5CE0638849
S31508000E30002B59D111F07F0F07D000F0B9FDD5F876
S31508000E40E4359B682846214698472846FFF79CFDC7
S31508000E504AE02146FFF7DAFD46E090F81231022B08
S31508000E6002D0032B06D03CE011F07F0F3CD000F0F7
S31508000E707FFD39E012F0800F16D001F07F0101EBFB
S31508000E80810100EBC10191F81E3133B140F23033D4
S31508000E90C2F2000301221A601AE040F23033C2F2AD
S31508000EA0000300221A6013E001EB810100EBC10187
S31508000EB091F8763333B140F23033C2F2000301229F
S31508000EC01A6005E040F23033C2F2000300221A60CD
S31508000ED0284640F23031C2F200010222FFF72EFD09
S31508000EE002E02146FFF792FD002038BD70B40646A1
S31508000EF000B3037843B1044600230133DBB214F888
S31508000F00015F002DF9D100E000235B000233138056
S31508000F100B7003234B70327862B1304602230025EA
S31508000F205C1CE4B2CA540233DBB20D5510F8012F2B
S31508000F30002AF5D170BC704770B582B0054600230B
S31508000F4001930320FFF792FBEB681A6901924FF4AD
S31508000F505464C0F20304032607E03046FFF786FB15
S31508000F60EB681A690192013C1CD0019A002AF4DA4E
S31508000F70019A42F001020192019A1A61EB681B6913
S31508000F8001934FF45463C0F2030304E0EA6812695C
S31508000F900192013B03D0019A12F0010FF6D103200A
S31508000FA0FFF764FB002002B070BD00BF10B4C47820
S31508000FB06CB9033300EB8200D0F8D0409B1006D002
S31508000FC0002251F8040B206001329342F9D1002027
S31508000FD05DF8044B704700BF70B40332D0F8D06098
S31508000FE0951009D00A460023346842F8044B0133A9
S31508000FF09D42F9D101EB8501084670BC704700BFD8
S3150800100070B40023C37001238370402383800129B1
S315080010100DD10123C37208230370042343704FF4D0
S31508001020A073C380022303724FF0A0450EE000258B
S3150800103061B90023C3720C230370062343704FF46F
S31508001040A063C3800025C4F20405FFE7C56005F563
S3150800105000630361467866B105F510620346002110
S315080010609A6102F500745C650131203204338E42C0
S31508001070F6D805F58063436105F58863C0F8CC307A
S315080010800678D6B1344605F5A06102460023C2F8B3
S3150800109090100133203104329C42F8D86EB105F520
S315080010A0805305EB063101F580510246C2F8D0306F
S315080010B003F5805304328B42F8D105F56065C0F814
S315080010C00C51002070BC704738B504460025037AD9
S315080010D0012B21D1C268936B6FF31043417A09B192
S315080010E043F480139363E268D3686FF386136FF350
S315080010F096536FF351436FF3D343D3602046FFF7FC
S315080011001BFFE378012B25D1052363F3440545F03E
S315080011102005E3689D6012E0C268D36843F0400387
S31508001120D360FFF709FF637A002B0CBF4FF45023F7
S315080011304FF4E813E26893631420FFF7A3FAE37801
S31508001140012B07D1E3689D68052262F3440545F043
S3150800115020059D60002038BDC3689A6842F00102E8
S315080011609A600020704700BFC3689A6822F001029F
S315080011709A600020704700BF00B583B00023019332
S31508001180019B43F020030193019B61F38A130193AA
S31508001190C368019A1A61C3681B6901934FF45463C3
S315080011A0C0F2030304E0C26812690192013B03D04E
S315080011B0019A12F0200FF6D10320FFF757FA002004
S315080011C003B05DF804FB00BF00B583B000230193AC
S315080011D0019B43F010030193C368019A1A61C3681F
S315080011E01B6901934FF45463C0F2030304E0C26819
S315080011F012690192013B03D0019A12F0100FF6D141
S315080012000320FFF733FA002003B05DF804FB00BFA4
S3150800121008B5C268D3686FF35D736FF39E730129CF
S3150800122008BF43F0005302D009B943F08043D360A6
S315080012303220FFF727FA002008BD00BFC3685B69A4
S3150800124013F0010F14BF002001207047C3685A69C4
S3150800125098691040704700BF03691A6861F3010274
S315080012601A60704710B40023C2689361C1686FF0B2
S3150800127080424A61C1684FF0FF344C60C1684A61D8
S315080012804FF40062C8F20002C1688A61C2789A42C5
S3150800129008BF102343F0804343F4701343F46053AC
S315080012A043F00C03C26891690B43936100205DF813
S315080012B0044B704770B5044600252E46D0F80C310D
S315080012C01D6003691A6865F3CC221A60C37A012B7C
S315080012D026D10321FFF7C0FFE2688023536220224C
S315080012E062F31F4563F30F05E1688D62A02161F380
S315080012F00F0663F31F46E368C3F804614FF490735F
S3150800130063F30F0662F31F46E368C3F808614FF4F8
S31508001310A07363F30F066FF31F46E368C3F80C6107
S3150800132020461021FFF728FF2046FFF74DFF2269C8
S31508001330002313612269536122694FF0FF319161DD
S315080013402269D3616378002B2CD0234600221646E7
S31508001350FF2599690868C00F002814BF4FF0904010
S315080013600020086099690E6199698D60013261787B
S3150800137004339142EDD8A9B1234600221646FF252B
S31508001380596D0868C00F002814BF4FF09040002020
S315080013900860596D0E61596D8D60013204336178AC
S315080013A09142EDD823691A6942F480721A61E3788A
S315080013B0012B09D10323402262F38A0343F48033C5
S315080013C062F35943226913632046FFF74BFF002057
S315080013D070BD00BF03699B68C3F34103022B05D0A8
S315080013E0032B05D0012B03D003207047012070473B
S315080013F0022070470369996883691A68C1F3410135
S31508001400022912BF6FF30A02032161F30A021A6066
S3150800141003695A6842F480725A600020704700BF18
S3150800142030B400224B78012B0B7800EB830401BF04
S31508001430A469012505FA03F363F30F021FBF646D60
S31508001440012505FA03F363F31F42236813F4004FDB
S315080014500DD18D6865F30A03CD7865F39343C98882
S3150800146061F3995343F0805343F4004323600369BF
S31508001470D9690A43DA61002030BC704730B40023CA
S315080014801A464C78012C097800EB810401BFA4693F
S31508001490012505FA01F161F30F021FBF646D0125ED
S315080014A005FA01F161F31F426FF3CF332360036935
S315080014B0D96921EA0202DA61002030BC704700BF10
S315080014C070B50B464A78012A53D10A7800EB820296
S315080014D091690A6809695C692CB96FF312010124DC
S315080014E064F3DC410DE064F312019D682C44013C71
S315080014F0B4FBF5F565F3DC41DC78012C08BF64F331
S315080015005E711C7800EB8404A4692161C178012905
S3150800151006D1197800EB81018C69196961610CE0C3
S31508001520D97801290CD0596999B101694D6B1C7894
S31508001530012606FA04F42C434C63D978012908D10C
S315080015400169896811F4807F0CBF42F0005242F0AD
S31508001550805242F00442197800EB810189690A60D9
S31508001560DA78012A41D1D9681A789B8AFFF71EFDD5
S315080015703BE00A7800EB8202516D0A6809695C69EA
S3150800158034B99C6864F31201012464F3DC410CE06D
S315080015909D682C44013CB4FBF5F4C4F3090464F3D8
S315080015A0DC4105FB04F565F312011C7800EB8404A5
S315080015B0646D2161C178012901BF197800EB8101A9
S315080015C04C6D196908BF6161D978012906D1597925
S315080015D011B142F0005201E042F0805242F004425A
S315080015E01B7800EB8300436D1A60002070BD00BFB6
S315080015F030B482B04B78012B49D1826913681469DB
S3150800160000944C696CB99DF800406FF306048DF898
S3150800161000409DF80240012565F3C4048DF8024098
S3150800162017E08D68AC4281BF4D619DF8004065F3B7
S3150800163006048DF800409EBF9DF8005064F3060529
S315080016408DF800509DF80240012565F3C4048DF815
S315080016500240009C1461C478012C01BF0C7800EB91
S315080016608404A5690C6908BF6C6143F004431360E0
S31508001670C378002B49D14B69002B46D00369586BB8
S315080016800A78012101FA02F202435A633DE00B7817
S3150800169000EB83035A6D1368126900924A6972B99E
S315080016A08C689DF8002064F306028DF800209DF8EA
S315080016B00220012464F3C4028DF802200EE08C682F
S315080016C04C619DF8002064F306028DF800209DF811
S315080016D00220012464F3C4028DF802200A7800EB84
S315080016E08202546D009A2261C278012A01BF0A78E3
S315080016F000EB8202546D0A6908BF626143F0044335
S315080017000A7800EB8200426D1360002002B030BCFC
S31508001710704700BF4B78012B0CD10B7800EB830088
S3150800172082691368002BB8BF43F0804343F4001363
S31508001730136007E00B7800EB8300426D136843F4EF
S3150800174000131360002070474B78012B0B7800EBD1
S3150800175083000CBF8269426D13686FF35553C978CD
S315080017600239C9B2012998BF43F08053136000209B
S31508001770704700BF03699A69D8691040000C704722
S3150800178000EB81014B6D9B680269506918407047F0
S3150800179003699869DB69184080B2704782B00023F4
S315080017A00093C0238DF803304FF00003012262F343
S315080017B0C4038DF8023018238DF80030436D009A63
S315080017C01A61C378012B08D1436D00F2CC525A61D5
S315080017D0436D1A684FF080221A6002B0704700BF46
S315080017E070B50446FFF70CFC012384F81231002378
S315080017F084F8143163787BB3234600220126114608
S31508001800402583F81D6183F81C21A3F8222183F85B
S315080018101F11C3F82451C3F82811C3F83011013237
S31508001820607828339042ECD8B0B12346002211469E
S31508001830402583F8751383F87423A3F87A2383F86D
S315080018407713C3F87C53C3F88013C3F8881301329F
S31508001850283360789042ECD82046FFF785FC20466E
S31508001860FFF732FC20460021FFF7D2FC2046FFF79F
S3150800187021FD2046FFF770FC70BD00BF38B511F09A
S31508001880800F0FD001F07F0404EB840500EBC5053B
S3150800189005F58E7185F81C4101254D708A60CB705F
S315080018A0CC800DE001F07F0404EB840500EBC50550
S315080018B005F55D7185F8744300244C708A60CB7019
S315080018C0022B04BF00230B71FFF7AAFD002038BDC9
S315080018D008B5CAB212F0800F01F07F0303EB830349
S315080018E000EBC30314BF03F58E7303F55D7301F0B4
S315080018F07F011970D2095A701946FFF7BFFD0020FB
S3150800190008BD00BF38B501F07F0404EB840500EB81
S31508001910C50505F55D71CA604B6100238B614B7087
S3150800192085F87443C378012B08BF0A6114B9FFF719
S315080019305FFE01E0FFF7C4FD002038BD70B501F079
S315080019407F0404EB840500EBC50505F58E710126B9
S315080019504E7085F81C41CA600A6100228A614B6193
S3150800196014B9FFF745FE01E0FFF7AAFD002070BD98
S3150800197010B5CAB212F0800F1FBF01F07F0303EB48
S31508001980830300EBC30303F58E7302BF01EB8103E8
S3150800199000EBC30303F55D7301249C7001F07F011E
S315080019A01970D2095A701946FFF7B4FE002010BD07
S315080019B010B5CAB212F0800F1FBF01F07F0303EB08
S315080019C0830300EBC30303F58E7302BF01EB8103A8
S315080019D000EBC30303F55D7300249C7001F07F01DF
S315080019E01970D2095A701946FFF7AEFE204610BD87
S315080019F0002361F30A13026911680B4313607047E9
S31508001A0008B503695A6842F002025A600320FEF7D5
S31508001A1039FE08BD2DE9F04F87B08146FFF70EFC69
S31508001A20002800F0A0824846FFF710FC83460028ED
S31508001A3000F09B8210F4002F08BF00205CD04846B7
S31508001A40FFF798FE0446002854D04D464F46002618
S31508001A5040F29C08C2F20008CDF800B0C34614F064
S31508001A60010F40D05FFA86FA48465146FFF788FECE
S31508001A70804610F0010F23D04FF001086B6DC3F8B4
S31508001A80088099F80330434508D16B6D1A69C2F38B
S31508001A901202D7F87C339B1AC7F88C33DBF8003070
S31508001AA01B6848465146984799F80330012B07D1D9
S31508001AB036B999F81131052B02D14846FFF76EFE63
S31508001AC018F0020F1FBF4FF002086B6D42469A606E
S31508001AD018F0080F07D0DBF800309B68484698478F
S31508001AE06B6D082098600136043528376408B6D12E
S31508001AF0DDF800B00120FFE71BF4802F00F0BC8062
S31508001B004846FFF745FE0646002800F0B4804F46D3
S31508001B10CA464FF0000840F29C02C2F20002019247
S31508001B20CDF808B0CDF8009016F0010F00F09780B8
S31508001B305FFA88F90098036919695C6B00EB8902FA
S31508001B409269926824FA09F4E401E4B20C43144059
S31508001B5014F0010F1CD0596B012202FA08F021EA91
S31508001B60000159631446BB699A60019A13685B6859
S31508001B700098494698470098C378A34208D1B8F117
S31508001B80000F05D190F81131042B01D1FFF706FE9D
S31508001B9014F0080F1EBF0824BB699C6014F0100FD0
S31508001BA01EBF1024BB699C6014F0400F1EBF402462
S31508001BB0BB699C6014F0020F1EBF0224BB699C60BF
S31508001BC014F0800F4BD05446DAF83021DAF8343165
S31508001BD0D01ADAF82431BB46BA69916989B29842B3
S31508001BE038BF03460333B1EB930F34D9DAF83451CF
S31508001BF0DAF83031AB422ED96BB30396009E5D1BE3
S31508001C00D4F82421AA4238BF15463046D4F82811FC
S31508001C104A46ABB2FFF7CAF9D4F828312B44C4F8C0
S31508001C202831D4F834312B44C4F83431DBF8183071
S31508001C309B6903359BB2B3EB950F09D9D4F8345198
S31508001C40D4F83031AB4205D9002BD8D1039E02E037
S31508001C50039E00E0039EDBF8183080229A6008F1A4
S31508001C60010804370AF1280A76087FF45DAFDDF823
S31508001C7008B0DDF8009001201BF0020F1EBFD9F84E
S31508001C800C3002225A61BBF1000F1FDA99F80A30AC
S31508001C9043B1D9F80C316FF341036FF30003D9F858
S31508001CA00C211360D9F810305A6822F001025A60E4
S31508001CB040F29C03C2F200031B689B69484698479A
S31508001CC0D9F80C304FF000425A6101201BF4006F1E
S31508001CD03AD000238DF8173099F812318DF817305D
S31508001CE040F29C03C2F200031B685B6948469847AA
S31508001CF0D9F810309968D9F80C304FF400625A6157
S31508001D0099F80A30FBB111F0010F1CD099F815317A
S31508001D10012B18D19DF81730DBB2032B13D1D9F854
S31508001D200C311A6842F001021A60D9F80C311A68A7
S31508001D3042F003021A604FF46D43CEF200031A69AB
S31508001D4042F006021A6101201BF0080F0CD040F27F
S31508001D509C03C2F200031B68DB6848469847D9F81B
S31508001D600C3008225A6101201BF0100F38D0D9F820
S31508001D700C309A6922F010029A61D9F80C301C6A64
S31508001D8004F00F0303EB830309EBC30505F55D7543
S31508001D90C4F34343022B02D0062B0FD019E0C4F339
S31508001DA00A14B4B14846E9682246FFF715F9EB6804
S31508001DB02344EB60AB692344AB610AE0484609F269
S31508001DC0CC510822FFF708F9C4F30A14AB69234477
S31508001DD0AB61D9F80C309A6942F010029A61012079
S31508001DE01BF4805F4CD00024274626462546D9F8A2
S31508001DF010305A6822F001025A6048462146FFF719
S31508001E00BBF999F8013063B14B462246FF21986920
S31508001E108160586D81600132043399F8010082426D
S31508001E20F5D3D9F810304FF0FF329A614FF0010818
S31508001E3068F30F0468F31F44D9F81030DC6147F0E3
S31508001E400B07D9F810305F6146F00B06D9F8103049
S31508001E501E61D9F810301A686FF30A121A604846DC
S31508001E60FFF79CFC45F48055D9F80C305D6140F2CB
S31508001E709C03C2F200031B681B6948469847404604
S31508001E801BF4005F26D04846FFF7B4FAD9F80C30A1
S31508001E90DC684846FFF79EFA032801BF002389F845
S31508001EA002304FF40073A9F804300FBF0923012349
S31508001EB089F8023040231CBFA9F80430052363F3D0
S31508001EC08D24D9F80C30DC60D9F80C304FF4005268
S31508001ED05A6101201BF4801F0DD040F29C03C2F208
S31508001EE000031B68DB6948469847D9F80C304FF45D
S31508001EF080125A6101201BF4001F0DD040F29C038A
S31508001F00C2F200031B681B6A48469847D9F80C308A
S31508001F104FF400125A6101201BF0804F0DD040F299
S31508001F209C03C2F200031B685B6A48469847D9F8C7
S31508001F300C304FF080425A6101201BF0040F15D077
S31508001F40D9F80C305C6814F0040F07D040F29C03F3
S31508001F50C2F200031B689B6A48469847D9F80C30BA
S31508001F605C60012002E0002000E0002007B0BDE828
S31508001F70F08F00BF08B54FF43053C4F201035B6B12
S31508001F8013F0450F07D14FF43052C4F20102536BD8
S31508001F9013F0450FFBD013F0040F04D0042001F012
S31508001FA0E1FF032008BD13F0010F04D0012001F062
S31508001FB0D9FF012008BD40F2FF5001F0D3FF0020F1
S31508001FC008BD00BF10B504464FF43053C4F20103F0
S31508001FD05B6B13F0450F07D14FF43052C4F2010280
S31508001FE0536B13F0450FFBD013F0040F04D00420F5
S31508001FF001F0B8FF032010BD13F0010F04D0012033
S3150800200001F0B0FF012010BD01F064FFA04249D1E4
S3150800201040F2FF5001F0A6FF002001F063FF4EF2E8
S315080020200803CFF6FF530340002B3DD000283DDBC5
S3150800203010F0804F3CD110F0005F3BD110F0805F6C
S315080020403AD110F0006F39D110F0806F38D110F006
S31508002050807F37D110F4000F36D110F4800F35D1B8
S3150800206010F4001F34D110F4801F33D110F4002F60
S3150800207032D110F4802F31D110F4003F30D110F452
S31508002080803F2FD110F4004F2ED110F4804F2DD160
S3150800209010F4005F2CD100F00800002814BF1A20A5
S315080020A0002010BD102010BD002010BD1C2010BD42
S315080020B0092010BD0A2010BD0B2010BD0C2010BD34
S315080020C00D2010BD0E2010BD0F2010BD102010BD14
S315080020D0112010BD122010BD132010BD142010BDF4
S315080020E0152010BD162010BD172010BD182010BDD4
S315080020F0192010BD2DE9F04182B00446002001F0F8
S31508002100F1FE10F0007F18BF0E2040F01781002264
S315080021100092019240F2F030C2F2000008210160FC
S315080021201025456040218160C2604FF480620261DB
S3150800213001F0B8FE2846FFF745FF002840F0FC806E
S3150800214040F2F030C2F2000040F29432C2F20002CD
S315080021501268AA4002603725456040228260002244
S31508002160C2604FF48062026101F09CFE2846FFF7C8
S3150800217029FF002840F0E18040F23C30C2F200001E
S315080021804FF0FF3303600823436030238360022344
S31508002190C360002505610123436101F0B1FE40F2E9
S315080021A0F030C2F2000005603326466040228260A5
S315080021B0C5604FF48062026101F074FE3046FFF795
S315080021C001FF002840F0BA80ADF104084FF43055FD
S315080021D0C4F2010540F22A664FF4001707E03846B4
S315080021E001F0B6FE18B101F0A3FE48F8040F6B6BB8
S315080021F03342F4D0082001F0ABFE20B1082001F0EC
S31508002200B1FE04209AE0022001F0A2FE20B10220CD
S3150800221001F0A8FE022091E0202001F099FE20B1ED
S31508002220202001F09FFE062088E04FF4007001F0A0
S315080022308FFE28B14FF4007001F094FE07207DE070
S3150800224040F2FF5001F08EFE009A130643EA12632D
S3150800225002F47F4143EA012302F47F0243EA122390
S31508002260012C34D113F4802F08BF252066D040F204
S31508002270F030C2F2000040F29432C2F20002126854
S315080022801204026037244460402282600022C26041
S315080022904FF48062026101F005FE2046FFF792FEC8
S315080022A0002847D140F2F030C2F200000222026054
S315080022B006244460402282600022C2604FF4806295
S315080022C0026101F0EFFD2046FFF77CFE36E013F4CD
S315080022D0803F08BF252031D040F2F030C2F200001E
S315080022E040F29432C2F200021268120402603724E5
S315080022F04460402282600022C2604FF4806202611C
S3150800230001F0D0FD2046FFF75DFEA0B940F2F0309F
S31508002310C2F2000000220260062444604021816067
S31508002320C2604FF48062026101F0BCFD2046FFF7EF
S3150800233049FE03E002E001E000E0FFE702B0BDE885
S31508002340F08100BF00B583B001238DF807304FF444
S315080023500060C4F202004FF4006101F075FC10B988
S3150800236000238DF807309DF8070003B05DF804FBDD
S315080023702DE9F04782B000248DF8074040F27C3002
S31508002380C2F2000076230375046044608460C4606A
S31508002390046101F059FD032001F076FD012001F0EA
S315080023A06DFD40F2F030C2F20000046044608460C3
S315080023B0C4604FF48063036101F074FD4FF4803408
S315080023C0802501E0013C0CD0284601F0C1FD00281B
S315080023D0F8D003233CB140F2FF5001F0C3FD0023BF
S315080023E001E00323FFE78DF807309DF8073013F067
S315080023F0FF0F03D09DF80700C0B2F5E040F2F030B9
S31508002400C2F200004FF4D5730360082343604023EB
S3150800241083600023C3604FF48063036101F042FDCB
S315080024204FF43053C4F201035A6B12F0450F0ED124
S315080024304FF480334FF43051C4F20101013B4A6B2B
S3150800244012F0450F02D1002BF8D103E013B112F0B8
S31508002450040F04D0042001F085FD032309E012F0DF
S31508002460400F08BF002304D0402001F07BFD002365
S31508002470FFE78DF807309DF8073013F0FF0F08D1F6
S3150800248040F26433C2F2000301221A604FF080451D
S3150800249014E040F2F030C2F200000025056037244F
S315080024A0446040228260C5604FF48062026101F098
S315080024B0F9FC2046FFF786FD8DF8070040F2F0305C
S315080024C0C2F2000000220260372444604021816085
S315080024D0C2604FF48062026101F0E4FC2046FFF717
S315080024E071FD8DF807009DF8073013F0FF0F78D1BE
S315080024F0002740F2F034C2F20004B846B94645F067
S31508002500004545F4801A4FF43055C4F20105C4F865
S315080025100090372666604023A360C4F80C904FF4F9
S3150800252080632361204601F0BDFC3046FFF74AFD73
S315080025308DF807009DF8073013F0FF0F03D09DF8BC
S315080025400700C0B250E0C4F800A029236360402306
S31508002550A360C4F80C804FF480632361204601F021
S31508002560A1FC6B6B13F0450F03D16B6B13F0450F92
S31508002570FBD013F0040F04D0042001F0F3FC03236E
S3150800258004E040F2FF5001F0EDFC43468DF80730B9
S315080025909DF8073013F0FF0F03D09DF80700C0B26F
S315080025A022E0404601F09EFC013701464FF6FE73D5
S315080025B0C043C00F9F4288BF00200028A7D19F4272
S315080025C006D91B238DF807309DF80700C0B20BE02B
S315080025D011F0804F1FBF40F26433C2F2000302229B
S315080025E01A609DF80700C0B202B0BDE8F08700BFC8
S315080025F038B501F04FFC002800F0BC8040F2643387
S31508002600C2F200031B68042B00F0B68040F2F030DB
S31508002610C2F200000023036002224260C0228260E8
S31508002620C3604FF48063036101F03CFCFFF7A2FC32
S31508002630002840F0A38001F055FC40F26834C2F24D
S3150800264000042060042001F04DFC6060082001F0C1
S3150800265049FCA0600C2001F045FCE06040F26433C0
S31508002660C2F200031B68062B18BF022B88BF012283
S315080026704AD840F2F030C2F2000000230360032279
S31508002680426040228260C3604FF48063036101F0B8
S3150800269009FC4FF43053C4F201035B6B13F0450F8A
S315080026A007D14FF43052C4F20102536B13F0450FB1
S315080026B0FBD013F0040F04D0042001F053FC0320D0
S315080026C038BD13F0010F04D0012001F04BFC0120A6
S315080026D038BD01F0FFFB032854D140F2FF5001F04A
S315080026E041FC002001F0FEFB10F4604F08BF020C0D
S315080026F00AD010F4005F47D110F4804F46D110F489
S31508002700004F45D10122FFE740F26433C2F20003CD
S315080027101B68042B33D040F29433C2F200031A60CC
S3150800272040F2F030C2F2000012040260092343604E
S31508002730C02383600023C3604FF48063036101F004
S31508002740B1FBFFF717FC0546D8B901F0CBFB40F201
S315080027505434C2F200042060042001F0C3FB606018
S31508002760082001F0BFFBA0600C2001F0BBFBE06075
S31508002770284638BD252038BD002038BD38BD002084
S3150800278038BD38BD102038BD132038BD102038BDDF
S315080027900F2038BDF0B4014640F26433C2F200039C
S315080027A01C6880F8564040F29433C2F200031B6856
S315080027B0A0F8543040F25433C2F200031A68150EDA
S315080027C0E8B286090E70C5F383054D7000F0030064
S315080027D08870C2F30740C870C2F307200871D2B2E6
S315080027E04A715B681A0E1201CA80C3F30742C88889
S315080027F080B240EA1210C88002F00F020A72C3F3D0
S315080028000720C2094A72C0F380128A72C0F34012C6
S31508002810CA72C0F300120A7300224A73012C42D806
S3150800282000F00300800208610A69DBB242EA83030A
S315080028300B6140F25433C2F200039868020ED3B219
S315080028400C6944EA93140C61C2F3C2020A7503F0D8
S3150800285007034B75C0F307435A098A75C3F3820207
S31508002860CA7503F003035B000B76C0F307200B7EE3
S3150800287043EAD0130B760F690A7E0E7AF6B2012365
S3150800288003FA06F60E65023203FA02F2D517A2FB20
S31508002890062306FB05337E1CA2FB064506FB0355ED
S315080028A0C1E9124524E0022C22D103F03F031B04A0
S315080028B00B6140F25433C2F2000398680B69020EAA
S315080028C043EA02230B610B69C0F3074213430B610A
S315080028D0C0F307200A690023013243F10003DB0431
S315080028E043EA5233D2048A64CB644FF400730B650F
S315080028F0C0F380134B7600F03F004000887640F224
S315080029005433C2F200031A7A887E40EAD2108876D7
S3150800291002F07F02CA76DA68130ED8B2C4090C77B9
S31508002920C3F341144C77C3F382038B7700F003009B
S315080029308000C877C2F30743C87F40EA9310C87778
S31508002940C3F3401081F82000002081F8210003F02D
S31508002950010381F82230C2F30723DC0981F82340FA
S31508002960C3F3801481F82440C3F3401481F825404A
S31508002970C3F3001481F82640C3F3810481F8274085
S3150800298003F0030381F82830C2F3460281F82920B0
S31508002990012481F82A4040F26833C2F200031A681B
S315080029A0150E81F82C50C2F307452D02CD85CD8D25
S315080029B0ADB2C2F307263543CD8512060A635A68B7
S315080029C00D6B160E45EA06450D630D6BC2F30746F9
S315080029D045EA06250D630D6BC2F3072635430D63DD
S315080029E0D2B281F834209A68150E81F83550C2F3B0
S315080029F007452D068D638D6BC2F3072645EA064506
S31508002A008D638D6BD2B245EA02228A63DB688A6BD4
S31508002A1042EA13628A63C3F3074291F83C5045EAD7
S31508002A20121581F83C5002F00F021202CA87CA8FAB
S31508002A3092B2C3F307252A43CA87C3F3460381F82C
S31508002A40403081F84140F0BC704700BF10B540F2F5
S31508002A506433C2F200031B68032B31D0022B31D832
S31508002A60B0F5805F30D0B0F5006F15D10120FFF7C3
S31508002A7041FB044650BB40F27C30C2F20000002203
S31508002A8002750260426082604FF40061C1600261B3
S31508002A9001F0DAF9204610BD0020FFF72BFB0446AB
S31508002AA0A8B940F27C30C2F200000022027502602A
S31508002AB042608260C260026101F0C6F9204610BD1C
S31508002AC0272010BD002010BD272010BD10BD10BD49
S31508002AD010B540F2F033C2F20003186007245C60B8
S31508002AE040229A600022DA604FF480621A61184622
S31508002AF001F0D8F92046FFF765FA10BD2DE9F04137
S31508002B0084B000268DF80F600C20012101F024F90D
S31508002B104FF40064C4F20204204608210C2201F096
S31508002B2099F8204609210C2201F094F820460A213A
S31508002B300C2201F08FF820460B210C2201F08AF8AE
S31508002B4020460C210A4601F085F84FF44067C4F286
S31508002B500207384602210C2201F07CF84FF4706314
S31508002B60019301258DF809504FF002088DF8088069
S31508002B708DF80A608DF80B50204601A901F01CF863
S31508002B800423019338460DEB030101F015F84FF4C1
S31508002B90805301938DF80B60204601A901F00CF8CB
S31508002BA04FF4006701978DF808808DF80B60204672
S31508002BB001A901F001F83846294601F003F94FF456
S31508002BC08000294601F0C8F801F032F9FFF7D0FB7A
S31508002BD08DF80F009DF80F3013F0FF0F03D09DF806
S31508002BE00F00C0B240E0FFF703FD8DF80F009DF817
S31508002BF00F3013F0FF0F03D09DF80F00C0B233E07B
S31508002C0040F27C30C2F20000002303750360436083
S31508002C108360C360036101F017F940F29830C2F28D
S31508002C200000FFF7B7FD8DF80F009DF80F3013F081
S31508002C30FF0F0BD140F29833C2F20003B3F85400E9
S31508002C4000040021FFF744FF8DF80F009DF80F30B0
S31508002C5013F0FF0F05D14FF40060FFF7F7FE8DF86C
S31508002C600F009DF80F00C0B204B0BDE8F08100BFA8
S31508002C702DE9F84307461646BDF8204040F239329A
S31508002C80C2F200020021117040F27832C2F200024C
S31508002C90116040F20440C2F2000001604FF4305265
S31508002CA0C4F20102D16240F26431C2F200010A683C
S31508002CB0022A02BF760A46EAC3564FF40074A046B3
S31508002CC040F2F030C2F20000046010224260402256
S31508002CD082600022C2604FF48062026101F0E2F86D
S31508002CE04FF48034802501E0013C04D0284601F0E9
S31508002CF02FF90028F8D01020FFF764F9002840F0D3
S31508002D00868040F23C30C2F200004FF0FF33036089
S31508002D10C0F80480902383600223C3600025056100
S31508002D200123436101F0ECF840F2F030C2F20000F2
S31508002D3006601124446040228260C5604FF48062B8
S31508002D40026101F0AFF82046FFF73CF9002860D190
S31508002D504FF43055C4F2010540F22A664FF4004894
S31508002D604FF000090BE0404601F0F2F838B14C4646
S31508002D7001F0DEF838510434202CF9D120376B6B7A
S31508002D803342F0D0082001F0E3F828B1082001F01A
S31508002D90E9F80420BDE8F883022001F0D9F828B143
S31508002DA0022001F0DFF80220BDE8F883202001F0B8
S31508002DB0CFF828B1202001F0D5F80620BDE8F88321
S31508002DC04FF4007001F0C4F84FF0FF344FF40015CB
S31508002DD058B14FF4007001F0C5F80720BDE8F88334
S31508002DE001F0A6F847F8040B013C284601F0B0F8B4
S31508002DF008B1002CF4D140F2FF5001F0B3F840F2CC
S31508002E00CC03C2F2000300201860BDE8F883BDE8D1
S31508002E10F883BDE8F88300BF2DE9F84F80461446CD
S31508002E20BDF8282040F23930C2F2000000210170B6
S31508002E3040F27830C2F20000016040F20440C2F26B
S31508002E40000001604FF43050C4F20100C16240F244
S31508002E506431C2F200010968022902BF640A44EA21
S31508002E60C3544FF40072164640F2F030C2F2000026
S31508002E70026010254560402282600022C2604FF43D
S31508002E808062026101F00EF82846FFF79BF80028D9
S31508002E9040F08B8040F2F030C2F200000460182443
S31508002EA04460402282600022C2604FF48062026160
S31508002EB000F0F8FF2046FFF785F8002877D140F2A2
S31508002EC03C30C2F200004FF0FF33036046609023A7
S31508002ED083600024C46004610123436101F010F893
S31508002EE0A3464FF43054C4F2010440F21A654FF475
S31508002EF0804625E0304601F02BF808B3CBF5007A7A
S31508002F00BAF11F0F10D85FEA9A0A19D0C1460027EE
S31508002F1059F8040B01F014F801375745F8D14FEA70
S31508002F208A0AD044D3440BE0002758F8070001F07A
S31508002F3007F80437202FF8D108F120080BF1200BE9
S31508002F40636B2B42D6D0082001F002F828B108207E
S31508002F5001F008F80420BDE8F88F022000F0F8FF19
S31508002F6028B1022000F0FEFF0220BDE8F88F1020ED
S31508002F7000F0EEFF28B1102000F0F4FF0520BDE8B0
S31508002F80F88F4FF4007000F0E3FF30B14FF4007093
S31508002F9000F0E8FF0720BDE8F88F40F2CC03C2F244
S31508002FA0000300201860BDE8F88FBDE8F88FBDE87B
S31508002FB0F88F00BF38B50546F8B140F2F030C2F2D6
S31508002FC0000040F29432C2F2000212681204026053
S31508002FD00D244460402282600022C2604FF4806261
S31508002FE0026100F05FFF2046FEF7ECFF044630B9A9
S31508002FF000F078FF2860204638BD262038BD38BD49
S3150800300000B583B000230193FFF79CF9012818BF88
S31508003010FF2008D101A8FFF7CDFF18B90198C0F322
S31508003020432000E0FF2003B05DF804FB08B5FFF776
S31508003030E7FF042804D0FF2814BF0120022008BD9A
S31508003040002008BD00B597B0FFF758FD60B940F2FB
S31508003050D003C2F200031A7802F0FE021A7068461C
S31508003060FFF798FB002006E040F2D003C2F2000307
S3150800307001221A70032017B05DF804FB08B540F268
S31508003080D003C2F2000301221A7050B9FFF7CEFF2F
S3150800309038B940F2D003C2F200031A7802F0FE02F1
S315080030A01A7040F2D003C2F20003187808BD00BFB8
S315080030B02DE9F043ADF5037D88461746D0B11CE0EF
S315080030C0013BDCB24FF000094FF40075E619009594
S315080030D002A872024B46FFF7CBFD80B9FFF7A6FFA1
S315080030E00128FBD008EB442002A92A4606F0D8F9A5
S315080030F04CB906E001204BB1E2E7012006E00120C9
S3150800310004E0002002E0013CE4B2DFE70DF5037DB0
S31508003110BDE8F0832DE9F043ADF5037D0F469046F3
S31508003120F0B120E0013BDCB24FF400754FF0000926
S3150800313002A807EB44212A4606F0B2F904EB080672
S31508003140009502A872024B46FFF766FE052818BFCF
S3150800315000280AD1FFF76AFF0128FBD04CB906E020
S3150800316001204BB1DEE7012006E0012004E0002043
S3150800317002E0013CE4B2DBE70DF5037DBDE8F08330
S3150800318010B596B0144640F2D003C2F200031B787D
S3150800319013F0010F18BF032021D103291AD8DFE83D
S315080031A001F002041015002019E0A8B96846FFF7D7
S315080031B0F1FA129B5B0A139A43EAC2532360002072
S315080031C00DE04FF400731380002008E030B9202387
S315080031D0136004E0042002E0002000E0002016B09E
S315080031E010BD00BF0020C4F2AA20704708B54FF0F2
S315080031F00070012100F0F8FD4FF00070002100F08A
S31508003200F3FD08BD0023036043608360C360036168
S3150800321043618361C361036243628362C36203637A
S3150800322043638363C3634022026420224264836447
S31508003230C364036543658365C36503668022426686
S315080032408366C366036743678367C3674FF0806215
S31508003250C0F880204FF00072C0F884204FF08071CB
S31508003260C0F888104FF40011C0F88C10C0F89030E0
S31508003270C0F89430C0F89830C0F89C30C0F8A03038
S31508003280C0F8A420C0F8A8304FF40032C0F8AC202B
S315080032904FF48072C0F8B020C0F8B430C0F8B83027
S315080032A0704700BF82B0002301934FF40043C4F275
S315080032B002031A6902F01C02890101F4F8610A4343
S315080032C0C00281B20A4342F001021A614FF4004279
S315080032D0C4F202024FF6FE71C0F20401019B0133EB
S315080032E00193136913F0010F02D0019B8B42F5D9A4
S315080032F0019A4FF6FF73C0F204039A421FBF4FF4B8
S315080033000043C4F20203586980B208BF002002B025
S31508003310704700BF10B483B0002301934FF40043F5
S31508003320C4F202031C6904F01C0444F00304890176
S3150800333001F4F8610C43C00281B20C435A611C6166
S315080033404FF40042C4F202024FF6FE71C0F20401C5
S31508003350019B01330193136913F0010F02D0019BFE
S315080033608B42F5D901984FF6FF73C0F20403C01AD1
S3150800337018BF012003B05DF8044B7047F0B587B05D
S3150800338004460D460023059300934FF40043C4F208
S3150800339002031E6926F01C0601A800F06FFC0299BC
S315080033A04FF45343CFF6CE630B444EF2BF12C0F22E
S315080033B0E402934298BF46F008061AD94FF2401322
S315080033C0CFF6E9530B4447F63F02C0F27D1293420B
S315080033D098BF46F00C060CD94FF4F243CFF66C436F
S315080033E00B444FF4B442C0F26222934288BF46F0BF
S315080033F004064FF40043C4F202031E612846002166
S315080034004FF40042FFF786FF002800F00F814FF0C7
S3150800341080630593059B2BB1059B013B0593059B93
S31508003420002BF9D12368002B5ED001274FF6FE76D4
S31508003430C0F20406009B0133009328463946FFF77D
S3150800344031FF00F0040083B213B9009BB342F1D9EF
S31508003450009A4FF6FF73C0F204039A4208BF002091
S3150800346000F0E9800021009128464FF48052FFF7CA
S3150800347051FF002800F0DC8001274FF6FE76C0F2E7
S315080034800406009B0133009328463946FFF70AFFD6
S3150800349000F0200080B210B9009BB342F1D9009A1F
S315080034A04FF6FF73C0F204039A4208BF002000F0EB
S315080034B0C2800023009328461021FFF7F3FE00F090
S315080034C004039BB21BB14FF40063236201E000239F
S315080034D0236200F002039BB213B1002363611BE071
S315080034E04FF48043636117E06369226AD20842EAAF
S315080034F053022846002192B2FFF70CFF002800F07D
S3150800350099806FF07F430593059B2BB1059B013B83
S315080035100593059B002BF9D14FF40043C4F202032F
S31508003520196848F20F12CFF620720A40A06861683F
S315080035300843E16808432169084361690843A169AA
S315080035400843E1690843216A0843616A0843A16A96
S315080035500843E16A0843216B0843616B01430A4348
S315080035601A60E16BA26B1143226C1143626C114322
S31508003570A26C1143E26C1143226D1143626D0A433A
S315080035805A60A26D9A60E26DDA609869A16E626E01
S315080035901143E26E1143226F1143626F11434FF6D6
S315080035A0417202400A43216E42EA01419961E16F84
S315080035B0A26F0A43DA6103F58053996943F62372C9
S315080035C0CFF6DE020A40D4F88400D4F88010084307
S315080035D0D4F888100843D4F88C100843D4F890100F
S315080035E00843D4F894100843D4F898100843D4F83C
S315080035F09C100843D4F8A01001430A439A61D4F8F2
S31508003600A410D4F8A820114341F40001D4F8AC2042
S315080036101143D4F8B0201143D4F8B8200A43D4F89B
S31508003620B41042EA81021A60012004E0002002E098
S31508003630002000E0002007B0F0BD00BF40B14FF405
S315080036400043C4F202031A6842F008021A6070477F
S315080036504FF40043C4F202031A6822F008021A6003
S31508003660704700BF40B14FF40043C4F202031A6822
S3150800367042F004021A6070474FF40043C4F2020392
S315080036801A6822F004021A60704700BF4FF410430C
S31508003690C4F202031A6842F001021A60704700BFBA
S315080036A04FF41043C4F20203186800F00100704793
S315080036B04FF41043C4F202039A6942F480129A61E5
S315080036C0704700BF40B14FF41043C4F202039A6931
S315080036D042F400529A6170474FF41043C4F2020351
S315080036E09A6922F400529A61704700BF40B14FF4BC
S315080036F01043C4F202039A6942F002029A617047C3
S315080037004FF41043C4F202039A6922F002029A6146
S31508003710704700BF08B50120FFF790FFFFF7C8FF05
S315080037200120FFF79FFF0120FFF7CCFF0120FFF7DD
S31508003730DDFF08BD2DE9F047B2B04FF0F05001218A
S3150800374000F00AFB4720012100F006FB4FF48040F9
S31508003750012100F037FB012000F00AFC8E2330938C
S3150800376000268DF8C66002248DF8C4408DF8C7601F
S315080037708DF8C5403746C4F20207384630A900F02E
S315080037801BFA384601210B2200F064FA3846214616
S315080037900B2200F05FFA384603210B2200F05AFA92
S315080037A0384607210B2200F055FA4FF40063309390
S315080037B08DF8C6608DF8C4408DF8C7608DF8C54091
S315080037C04FF4C057C4F20207384630A900F0F4F99E
S315080037D038460B210A4600F03DFA322330938DF81D
S315080037E0C6608DF8C4408DF8C7608DF8C5404FF4A3
S315080037F00068C4F20208404630A900F0DDF94046E8
S3150800380001210B2200F026FA404604210B2200F083
S3150800381021FA404605210B2200F01CFA4FF4C0435A
S3150800382030938DF8C6608DF8C4408DF8C7608DF862
S31508003830C540384630A900F0BFF938460D210B229D
S3150800384000F008FA38460E210B2200F003FAFFF7BB
S31508003850CDFCFFF71BFFFFF723FF0128FBD001A8CC
S31508003860FFF7D0FC0024019408944FF400730B93DF
S315080038700C944FF000430F9320231293149415943D
S3150800388016944FF4006309934FF4804306934FF060
S31508003890020A4FF003094CF2F108C0F2070841F298
S315080038A01967C0F22207A6B230465146FFF7FAFC5E
S315080038B060F31F4530464946FFF7F4FC60F30F05F1
S315080038C0BD4218BF454503D00134202CEBD109E091
S315080038D0202C07D949F26C60C0F600004FF4A1719C
S315080038E004F0F0FE01A8A1B2FFF748FD38B949F285
S315080038F06C60C0F6000040F2471104F0E3FE42F2A5
S315080039008073C2F2000342F2D002C2F200029A6049
S31508003910DB6000221A605A604FF41041C4F20201BB
S315080039200B6141F68023C2F2000341F69020C2F2F1
S31508003930000098601A60DB605A6040225A719A88C3
S315080039404FF4C86060F30C029A808022DA70CB606C
S31508003950FFF7E0FE32B0BDE8F08700BF40F21C6317
S31508003960C2F2000308221A7000225A7027229A709F
S315080039706922DA705B221A7145225A71704700BFB4
S3150800398038B541F68023C2F20003DB78DB091DD186
S3150800399041F68024C2F200046588C5F30D0542F697
S315080039A02000C2F2000041F69021C2F200012A4628
S315080039B005F076FDE37843F08003E3704FF4104397
S315080039C0C4F2020301229A60284638BD002038BD99
S315080039D038B542F28073C2F20003DB78DB0900D007
S315080039E0FEE742F29073C2F200031D8842F2D00449
S315080039F0C2F20004204642F62001C2F200012A461D
S31508003A0005F04EFD42F28073C2F200039C6000226C
S31508003A101A60102199705A60C5F30B059D80B02273
S31508003A20DA704FF41043C4F2020301225A6038BD1B
S31508003A304FF47053C4F202031B69002B0DDA4FF4DE
S31508003A407053C4F2020340F22312C4F267525A605A
S31508003A5048F6AB12CCF6EF525A6070474FF47053E3
S31508003A60C4F202031A6942F000421A61704700BFA5
S31508003A704FF47053C4F20203D86070474FF4705382
S31508003A80C4F20203DB6813F4803F1BD14FF4705372
S31508003A90C4F20203DB6813F0100F15D14FF470530C
S31508003AA0C4F20203DB6813F0EF0F0FD14FF4705323
S31508003AB0C4F20203D86800F0020000280CBF0820F0
S31508003AC00720704701207047052070470620704779
S31508003AD000B583B008238DF80730FFF7CFFF8DF8C0
S31508003AE007009DF80730DBB2012B08D1FFF7C6FFA8
S31508003AF08DF807009DF80730DBB2012BF6D09DF84C
S31508003B00070003B05DF804FB70B50546002659B1F9
S31508003B10012908BF4FF4807606D0022914BF4FF456
S31508003B2040764FF40076FFE7FFF7D2FF082821D149
S31508003B304FF47054C4F20204236923F440732361DA
S31508003B4023691E432661236923F0F8032361236949
S31508003B5043F002031D432561236943F4803323613F
S31508003B60FFF7B6FF236923F002032361236923F0D5
S31508003B70F803236170BD00BF70B505460E46FFF712
S31508003B80A7FF082816D14FF47054C4F2020423691B
S31508003B9023F440732361236943F400732361236983
S31508003BA043F0010323612E60FFF792FF236923F098
S31508003BB00103236170BD00BFF0B40023012503266D
S31508003BC005FA03F20C681440944238D107685A0083
S31508003BD006FA02F4E44327400760076891F804C030
S31508003BE00CFA02FC4CEA070707600F79013FFFB29F
S31508003BF0012F16D887683C40846087684C799440C2
S31508003C003C43846047689CB205FA04FC27EA0C0723
S31508003C104760476891F806C00CFA04F4A4B23C431E
S31508003C204460C7689CB2640006FA04F427EA0404F0
S31508003C30C460C468CF7907FA02F22243C26001332E
S31508003C40102BBDD1F0BC7047036919420CBF002088
S31508003C500120704710B401F007039B00C90800EB68
S31508003C608100046A0F21994024EA01010162016A70
S31508003C709A40114301625DF8044B704710B44FF443
S31508003C806053C4F202039B6803F00C03042B09D0AB
S31508003C90082B0DD0002B36D14FF41053C0F2F40385
S31508003CA0036035E04FF4D853C0F2B70303602FE042
S31508003CB04FF46053C4F202035C685A6802F03F028C
S31508003CC014F4800F4FF46053C4F202035B68C3F325
S31508003CD0881319BF4FF4D854C0F2B7044FF41054E0
S31508003CE0C0F2F404B4FBF2F101FB03F14FF46053A4
S31508003CF0C4F202035A68C2F3014201325200B1FB10
S31508003D00F2F3036004E04FF41053C0F2F4030360C7
S31508003D104FF46052C4F202029168C1F3031140F2F3
S31508003D20D403C2F20003595CC9B2046824FA01F14B
S31508003D3041609468C4F382241C5DE4B221FA04F459
S31508003D4084609268C2F342329B5CDBB2D940C160A0
S31508003D505DF8044B704700BF39B14FF46053C4F2A5
S31508003D6002031A6B1043186370474FF46053C4F28A
S31508003D7002031A6B22EA00001863704739B14FF440
S31508003D806053C4F202035A6B1043586370474FF4EA
S31508003D906053C4F202035A6B22EA00005863704764
S31508003DA039B14FF46053C4F202031A6C1043186415
S31508003DB070474FF46053C4F202031A6C22EA0000FB
S31508003DC01864704739B14FF46053C4F202035A6C51
S31508003DD01043586470474FF46053C4F202035A6C98
S31508003DE022EA00005864704739B14FF46053C4F2B0
S31508003DF002031A691043186170474FF46053C4F2FE
S31508003E0002031A6922EA00001861704739B14FF4B3
S31508003E106053C4F202035A6A1043586270474FF45B
S31508003E206053C4F202035A6A22EA000058627047D5
S31508003E3008B54FF400600121FFF7E8FF4FF4006072
S31508003E400021FFF7E3FF08BD10B44FF43053C4F266
S31508003E5001035C68416882681143C26811430268BD
S31508003E60114302690A4324F4FD4424F07F042243E3
S31508003E70017D0A435A605DF8044B704748F2A00377
S31508003E80C4F22523186070474FF43053C4F2010377
S31508003E90186070474FF43053C4F20103186800F0F5
S31508003EA00300704710B402684FF43053C4F201039C
S31508003EB09A60DC6824F4FF6424F007048268416889
S31508003EC01143C2680A43006902432243DA605DF877
S31508003ED0044B70474FF43053C4F201031869C0B25B
S31508003EE0704700BF82B00023019342F61443C4F220
S31508003EF0010303440193019B186802B0704700BF91
S31508003F0010B402684FF43053C4F201035A6242688F
S31508003F109A62DC6A24F0F704C26881681143026970
S31508003F200A43406902432243DA625DF8044B70474C
S31508003F304FF43053C4F20103D3F88000704700BF32
S31508003F404FF43053C4F20103C3F88000704700BF32
S31508003F504FF43053C4F201035B6B18420CBF0020C8
S31508003F60012070474FF43053C4F201039863704739
S31508003F70DC23C4F227231860704700BF30B585B02C
S31508003F8004460D46038A23F440531B041B0CCA88B7
S31508003F9013430382838923F4B05323F00C031B04D1
S31508003FA01B0C0989AA880A4369890A4392B21343F2
S31508003FB08381838A23F440731B041B0CAA89134349
S31508003FC083826846FFF75AFE4FF4A052C4F20102F4
S31508003FD04FF48053C4F201039C4218BF94420CBFAD
S31508003FE0039A029AA3891BB2002B02EB820202EB08
S31508003FF08202BDBF2B685B00B2FBF3F22968A4BF3F
S315080040008900B2FBF1F248F21F53C5F2EB13A3FB8A
S3150800401002135B091D01642003FB1023A08900B26B
S3150800402000280BDADB00323348F21F51C5F2EB11D8
S31508004030A1FB0321C1F3421129430AE01B013233D4
S3150800404048F21F51C5F2EB11A1FB0321C1F343113D
S31508004050294389B2218105B030BD00BF29B18389C2
S315080040609BB243F4005383817047838923F400533A
S315080040701B041B0C83817047C1F3080181807047BC
S315080040808088C0F308007047038819420CBF0020D7
S315080040900120704782B04FF46053C4F202031A68D5
S315080040A042F001021A6000229A60196821F08471B0
S315080040B021F48031196043F21001C2F200415960BF
S315080040C0196821F480211960DA60009201921A6851
S315080040D042F480321A604FF46052C4F20202136846
S315080040E003F400330193009B01330093019B1BB932
S315080040F0009BB3F5A06FF2D14FF46053C4F20203EC
S315080041001B6813F4003F14BF012300230193019B8E
S31508004110012B46D14FF46053C4F202031A6C42F0E5
S3150800412080521A644FF4E042C4F20002116841F466
S31508004130404111609A689A609A6842F400429A600F
S315080041409A6842F4A0529A6045F20C42C0F2407254
S315080041505A601A6842F080721A604FF46052C4F2CC
S315080041600202136813F0007FFBD04FF47053C4F2B9
S31508004170020340F205621A604FF46053C4F2020368
S315080041809A6822F003029A609A6842F002029A60DC
S315080041904FF46052C4F20202936803F00C03082B32
S315080041A0FAD14FF46D43CEF200034FF000629A60E5
S315080041B002B0704732B1821811F8013B00F8013B92
S315080041C09042F9D1704700BFCA7E8B7E43EA02232C
S315080041D00278032A01BF487D0A7D42EA002243EAA3
S315080041E002431846704700BF00F10B010023DA01AD
S315080041F042EA530310F8012B52FA83F3DBB28842E2
S31508004200F5D11846704700BF10B504460A464078EF
S3150800421004F134010123FEF74BFFD0BB94F8332297
S3150800422094F8323243EA022212B24AF65523CFF6FE
S31508004230FF739A422FD194F86D2094F86C301B04C2
S3150800424043EA026294F86A30134394F86B2043EA0F
S31508004250022222F07F4244F24613C0F254039A42E5
S315080042601BD094F8890094F888301B0443EA006050
S3150800427094F88630034394F8870043EA002020F038
S315080042807F4044F24613C0F25403C01A18BF0120F7
S3150800429010BD032010BD022010BD002010BD00BFB8
S315080042A02DE9F041044603791BB3056B00F1340789
S315080042B0407839462A460123FEF72CFFE0B9002349
S315080042C02371636A9D421AD3E26913449D4219D247
S315080042D0E678012E19D94FF00108E269154460788D
S315080042E039462A464346FEF715FF013E012EF4D10C
S315080042F00EE00020BDE8F0810120BDE8F081002035
S31508004300BDE8F0810020BDE8F0810020BDE8F0811D
S315080043100020BDE8F08100BF38B504460D46036BA2
S315080043208B420CD0FFF7BCFF58B9607804F1340112
S315080043302A460123FEF7BCFE28B9256338BD0020AE
S3150800434038BD012038BD012038BD00BF08B588B189
S3150800435003688BB1197889B1D988828891420FD1BF
S315080043605878FEF78BFE00F00100002814BF0320E2
S31508004370002008BD092008BD092008BD092008BD80
S31508004380092008BD2DE9F041154603681C78303C24
S31508004390092C00F2B5815A783A2A40F0B1810233E5
S315080043A0036000230B60002C40F0718140F20C631F
S315080043B0C2F200031C68002C00F06C810C602378A4
S315080043C08BB16078FEF75AFE10F0010F0BD1002D65
S315080043D000F0638100F00400C0B2002814BF0A2070
S315080043E00020BDE8F081002020706070FEF72AFEEC
S315080043F010F0010F40F054811DB110F0040F40F089
S31508004400528120460021FFF7FFFE012818BF00252C
S3150800441017D194F8F631002B00F0488194F8FD2165
S3150800442094F8FC311B0443EA026294F8FA31134308
S3150800443094F8FB5143EA052520462946FFF7E4FE92
S31508004440FFE7032800F03581002840F0358194F80D
S31508004450402094F83F3043EA02231BB2B3F5007FAD
S3150800446040F02D8194F84B0094F84A3053EA002026
S315080044700DD194F85B2094F85A301B0443EA026283
S3150800448094F85830134394F8590043EA0020E06141
S3150800449094F84410E1704B1EDBB2012B00F2128136
S315080044A094F84130A370002B00F00F815A1E1A426F
S315080044B040F00E8194F8466094F8452042EA0622B8
S315080044C0228112F00F0F40F0068194F8487094F894
S315080044D0476056EA07260DD194F8577094F8566047
S315080044E0360446EA076794F854603E4394F85570D4
S315080044F046EA072694F843C094F8427057EA0C2710
S3150800450000F0EC8001FB00FC07EB121161448E42BF
S31508004510C0F0E780761AB6FBF3F3002B00F0E480D0
S3150800452040F6F576B3428CBF022601264FF6F5789B
S31508004530434500F2E8800233A36125622F4467628F
S315080045402944E162032E13D1002A40F0D08094F862
S31508004550631094F86220120442EA016194F860201C
S315080045600A4394F8611042EA0122A2629B000EE017
S31508004570002A00F0BF806744A762022E0FBF5B00C7
S3150800458003225A4303F0010318BF03EB520303F255
S31508004590FF13B0EB532FC0F0B0804FF0FF33236109
S315080045A00023E360032E63D1637194F8652094F8C1
S315080045B0643043EA02222A446261607804F13401D5
S315080045C00123FEF775FD002852D194F8332294F89A
S315080045D0323243EA022212B24AF65523CFF6FF7365
S315080045E09A4245D194F8372094F836301B0443EAAA
S315080045F0026294F83430134394F8352043EA0222D1
S3150800460045F25223C4F261139A4231D194F81B221F
S3150800461094F81A321B0443EA026294F818321343D8
S3150800462094F8192243EA022247F27223C6F241138A
S315080046309A421DD194F8232294F822321B0443EAA5
S31508004640026294F82032134394F8212243EA0223A3
S31508004650E36094F81F2294F81E321B0443EA0262B0
S3150800466094F81C32134394F81D2243EA022323616B
S31508004670267040F20863C2F200031A88013292B229
S315080046801A80E280002020632071BDE8F0810B20AB
S31508004690BDE8F0810C20BDE8F0810020BDE8F0817E
S315080046A00320BDE8F0810A20BDE8F0810D20BDE8B1
S315080046B0F0810120BDE8F0810D20BDE8F0810D20D4
S315080046C0BDE8F0810D20BDE8F0810D20BDE8F08140
S315080046D00D20BDE8F0810D20BDE8F0810D20BDE874
S315080046E0F0810D20BDE8F0810D20BDE8F0810D2098
S315080046F0BDE8F0810D20BDE8F0810D20BDE8F08110
S3150800470000230B6052E60233A36125622F446762D9
S315080047102944E162032617E72DE9F0410D4601F128
S3150800472009020369002B5ED0416991F80C800B7869
S31508004730202B1BD00E46002408F00807FFB203E022
S3150800474016F8013F202B11D0052B08BFE52347B1EA
S31508004750A3F1410C5FFA8CFCBCF1190F9CBF203306
S31508004760DBB202F8013B0134082CE9D10B7A202B85
S3150800477022D0561C2E2313700B7A202B1BD001F146
S315080047800804171D324608F010085FFA88F603E099
S3150800479014F8013F202B0FD046B1A3F1410C5FFA64
S315080047A08CFCBCF1190F9CBF2033DBB202F8013B2D
S315080047B0BA42EDD100E03246CB7A2B72CC7F8B7FA2
S315080047C01B0443EA04630C7F23434C7F43EA042318
S315080047D02B604C7E0B7E43EA0423AB80CC7D8B7D1D
S315080047E043EA0423EB8000231370AE6946B3EB69F2
S315080047F033B3036900240BB3028C4FF6FF739A4256
S3150800480008BF00241AD0C769388890B10024A0468A
S31508004810414601F02BFC70B1EA69013AA2420CD973
S315080048200134321902F8010C37F8020F0028EFD1CB
S3150800483004E0002402E0002400E0002400233355AD
S31508004840BDE8F08110B50446FFF72AFD03460028A7
S3150800485054D12378032B49D16379002B46D0002302
S31508004860236304F1340104F50D700B46002203F8A6
S31508004870012B8342FBD1552384F83232AA2384F8CC
S315080048803332522384F8343084F83530612384F87F
S315080048903630412284F83720722084F8180284F8CA
S315080048A0190284F81A2284F81B32236984F81C3208
S315080048B0C3F3072284F81D221A0C84F81E221B0E45
S315080048C084F81F32E36884F82032C3F3072284F899
S315080048D021221A0C84F822221B0E84F823326078CF
S315080048E062690123FEF716FC0023637160780021D4
S315080048F00A46FEF745FC031C18BF0123184610BDDF
S3150800490002398369023B99423DBF8278C36A02FB3A
S3150800491001300020704700BFF8B505460C4601294E
S315080049205CD9836999425BD20378022B28D0032B82
S3150800493038D0012B56D101EB5106416A01EB5621BD
S31508004940FFF7EAFC002850D1C6F308032B4493F876
S3150800495034700136696A284601EB5621FFF7DCFCFC
S31508004960002845D1C6F30806354495F8340047EAC9
S31508004970002014F0010F14BF0009C0F30B00F8BDA6
S31508004980416A01EB1421FFF7C7FCA0BB640004F4DD
S31508004990FF742B1993F834302C4494F8350043EA05
S315080049A00020F8BD416A01EBD411FFF7B5FC28BB1E
S315080049B0A40004F4FE742B1993F8360093F83720F4
S315080049C0120642EA004293F8350042EA00202C44D7
S315080049D094F83430184320F07040F8BD0120F8BD33
S315080049E00120F8BD4FF0FF30F8BD4FF0FF30F8BD9D
S315080049F04FF0FF30F8BD4FF0FF30F8BD4FF0FF30F5
S31508004A00F8BD00BF70B504460D46E18081680129EE
S31508004A1038D003689A69914236D271B91A78032A4E
S31508004A2001D1996A49B90022E2601A89AA422DD9A8
S31508004A309B6A03EB151323611BE09E783601B5428A
S31508004A4010D32068FFF768FF0146B0F1FF3F1FD07B
S31508004A5001281FD923689B6998421DD2AD1BADB2A8
S31508004A60AE42EED9E1602068FFF74AFF00EB151069
S31508004A70206105F00F05236803EB451334336361A2
S31508004A80002070BD022070BD022070BD022070BDDE
S31508004A90012070BD022070BD022070BDF8B5054624
S31508004AA00C461646012998BF02237CD98369994288
S31508004AB028BF022377D20378022B40D0032B50D08D
S31508004AC0012B18BF02236BD101EB5107416A01EB99
S31508004AD05721FFF721FC0346002861D1C7F30803D5
S31508004AE014F001041FBFEA1892F8342002F00F02EE
S31508004AF0F1B21ABF42EA0112D2B2F2B22B4483F8DB
S31508004B003420013701232B71696A284601EB5721A6
S31508004B10FFF702FC0346002842D1C7F3080714B181
S31508004B20C6F3071607E0EA1992F8342022F00F02B6
S31508004B30C6F3032616432F4487F8346030E0416AEB
S31508004B4001EB1421FFF7E8FB034648BB640004F4B5
S31508004B50FF742A1982F83460C6F3072682F835608E
S31508004B601EE0416A01EBD411FFF7D6FB0346B8B93C
S31508004B70A40004F4FE742A1992F8371009062C4486
S31508004B8001F070410E4384F83460C6F3072182F8B9
S31508004B903510310C82F83610360E82F83760FFE78A
S31508004BA001222A71FFE71846F8BD00BF2DE9F0413A
S31508004BB00546884631B9C66876B183699E4228BFDC
S31508004BC001260AE0FFF7A8FE012847D9AB699842F3
S31508004BD028BF464601D24DE0012634460227013455
S31508004BE0AB699C4202D3012E3BD93C462846214656
S31508004BF0FFF792FE38B1B0F1FF3F18BF012833D056
S31508004C00B442ECD132E02646284621466FF070427F
S31508004C10FFF744FF0346D0F1010038BF0020B8F182
S31508004C20000F08BF002028B1284641462246FFF754
S31508004C3035FF03465BB9EE602B69B3F1FF3F18D029
S31508004C40013B2B6101236B712046BDE8F081012BE6
S31508004C5014BF01204FF0FF30BDE8F0810120BDE808
S31508004C60F0810020BDE8F081BDE8F0810020BDE8B4
S31508004C70F0812046BDE8F0812DE9F84304460E464A
S31508004C80C5880135ADB2002D6AD00369002B6AD0FC
S31508004C9015F00F075BD101330361C16821B90368B9
S31508004CA01B89AB4262D952E000688378013B13EA5C
S31508004CB015134CD1FFF730FE8046012859D9B0F1BB
S31508004CC0FF3F59D020688369984539D3002E56D0BE
S31508004CD0E168FFF76BFF8046002853D0012854D0BF
S31508004CE0B0F1FF3F54D02068FFF7DAFA002852D116
S31508004CF0236803F1340100231A46CA540133B3F575
S31508004D00007FFAD1266830464146FFF7F9FD306341
S31508004D1000264FF001090CE083F804902068FFF79D
S31508004D20BFFA00283AD123681A6B01321A63013692
S31508004D30F6B223689A78B242EED81A6B921B1A63B7
S31508004D40C4F80C8020684146FFF7DAFD2061E5804B
S31508004D50236803EB4713343363610020BDE8F88307
S31508004D600420BDE8F8830420BDE8F8830420BDE8E4
S31508004D70F8830220BDE8F8830120BDE8F883042003
S31508004D80BDE8F8830720BDE8F8830220BDE8F8836C
S31508004D900120BDE8F8830120BDE8F8830120BDE8BD
S31508004DA0F88300BF2DE9F04F89B005460021FFF7CB
S31508004DB029FE002840F0AC804FF0FF09C8464F4650
S31508004DC049F21471C0F60001029101F10C02049235
S31508004DD04FF6FF7A4FF0000B28682969FFF79CFA0F
S31508004DE0002840F096806C692678002E00F09280A4
S31508004DF0E37A03F03F02E52E7FD013F0080F04D0C4
S31508004E000F2A18BFB8467BD101E00F2A58D1EB69A3
S31508004E100193002B74D016F0400F06D094F80D902D
S31508004E2006F0BF06EB882B8403E0B04518BFB846EA
S31508004E3066D1617B0391494518BFB84660D123788E
S31508004E4023F04003013B03EB430203EB8202059286
S31508004E50029A02F1FF394FF001080796059E06955A
S31508004E604546DDF8108019F8013FE2185078E35CF2
S31508004E7043EA00207DB101F01FF90546FE2E56D8FB
S31508004E80731C0593019931F8160001F015F985424E
S31508004E904FD1059E01E050454DD1C145E3D1A84605
S31508004EA00596079E069D237813F0400F39D0B8F172
S31508004EB0000F36D0059A019931F812308BB33BE0D2
S31508004EC0B8F1000F04D12046FFF78EF9484523D0E4
S31508004ED0A5F820A0AB69DA7A12F0010F08BF04F131
S31508004EE00B0002D00BE0844218D014F8011B13F80B
S31508004EF0012B9142F7D0B84602E0B84600E0B84622
S31508004F0028465946FFF7B8FE00283FF465AF07E084
S31508004F1016E015E0042013E0002011E000200FE061
S31508004F200EE0013E5FFA86F8DDF80C90E8E7069D8C
S31508004F3002E0069D00E0069DDDF80C90B846DFE726
S31508004F4009B0BDE8F08F00BF2DE9F04F87B0814664
S31508004F5088460B782F2B18BF5C2B08BF01F1010878
S31508004F600023836098F800301F2B07D80021FFF72D
S31508004F7049FD03460022C9F814207AE14FF0010AD8
S31508004F8049F2806BC0F6000B49F28C61C0F600014D
S31508004F90049149F29462C0F60002059298F800302E
S31508004FA02F2B18BF5C2B08D108F10103984613F87C
S31508004FB0012B2F2A18BF5C2AF8D0D9F81C5098F86C
S31508004FC000002F2818BF1F282CD95C2800F02D8137
S31508004FD0AF1E4646544607E05C2B00F02881B2F522
S31508004FE0807F00F041811446514601F03FF80146A2
S31508004FF0002800F039817F2809D8222900F0348159
S315080050005A4612F8013F13B19842FAD12CE127F813
S31508005010021F621C16F8013F18462F2B18BF1F2BBC
S31508005020DAD801E00024524690441F2898BF042687
S3150800503001D90026FFE7002C00F0168104F1004391
S31508005040013B5A0035F813302E2B18BF202B40F0A1
S31508005050F080931C2B4407E033F8042C023B2E2ADD
S3150800506018BF202A40F0E580013CF5D1FCE003F8A2
S31508005070011B8342FBD12B88202B18BF2E2B40F017
S31508005080E48028460023013330F8021F202918BF80
S315080050902E29F8D0002B00F0D98046F00306D5E07B
S315080050A0013C05D10821039100220192029205E0F4
S315080050B0023A32F8021C2E29F2D1F3E75F1C35F8C2
S315080050C01300002861D0202808D0E31B18BF01234D
S315080050D02E2814BF002203F001021AB146F0030677
S315080050E03B46EBE7019A0399BC4218BF8A4214D3A0
S315080050F00B2903D146F00306029A49E00BB146F0A4
S315080051000306A74243D8029A9300DBB202932346CA
S315080051100B21039108220192D0E77F280DD900219F
S3150800512000F0A4FF0346002800F0A08005990B4470
S3150800513013F8800C46F0020650B101462B2807D01A
S31508005140049A12F8013F002B00F087809942F8D1A3
S3150800515046F003065F2010E0029A42F0020202922D
S315080051600BE0A0F161039BB2192B9FBF029B43F092
S3150800517001030293203898BF80B2D9F818300199F4
S3150800518058543B460131019198E7029A00E0029A89
S31508005190D9F818301978E52904BF05211970039B39
S315080051A0082B02BF9200D2B20292029901F00C03B8
S315080051B00C2B03D001F00302032A01D146F00206A4
S315080051C016F0020F0AD1029901F00302012A08BF5C
S315080051D046F01006042B08BF46F00806D9F8183022
S315080051E0DE724846FFF7DEFDD9F81830DA7A03464C
S315080051F048B104283DD102F00403DBB2002B14BFEA
S315080052000346052335E012F0040F32D1D9F81410FD
S31508005210CB7A13F0100F06D0D9F80000FEF7D4FFAA
S31508005220C9F80800BAE6052323E00024524690444C
S31508005230FFE66700EA194FF0000325F81430D9F89D
S31508005240183003F10B00202111E700232F4437F80B
S31508005250021C2E293FF426AF22E7A0F141039BB298
S31508005260192B7FF679AF7CE7062302E046F00206A3
S315080052706EE7184607B0BDE8F08F00BF2DE9F04F7E
S3150800528083B0044689464FF0FF0B5E460425D84690
S3150800529049F2147AC0F6000A0AF10C0300930027B3
S315080052A070E02068FFF738F8054600286ED1626975
S315080052B01378002B74D0D17AE52B18BF2E2B59D032
S315080052C001F03F01082914BF00200120484518BFF6
S315080052D0464651D10F2943D113F0400F06D092F814
S315080052E00DB003F0BF03E188218403E09E4218BF96
S315080052F0464641D192F80DE0DE4518BF46463BD1F9
S31508005300D4F81CC0117801F03F01013901EB4105C1
S3150800531001EB85050AF1FF3101260193DDF800B09E
S3150800532011F8013FD0184078D35C43EA002036B123
S31508005330FE2D32D82CF815000646013503E04FF647
S31508005340FF73984229D15945EAD1019B127812F088
S31508005350400F1ED0FE2D98BF2CF8157019D91CE0E9
S3150800536010461EB9FEF740FF58451BD04FF6FF738F
S31508005370238417E04646FFE720463946FFF77CFCBC
S31508005380054618B9216900298BD15DB1002323612F
S3150800539008E0013BDEB2F346EEE7F3464646EBE7A6
S315080053A00425F3E7284603B0BDE8F08F2DE9F04160
S315080053B00446C588018C4FF6FF73994208BF2946F3
S315080053C0FFF720FB0346D0B9E52701264FF0000872
S315080053D020682169FEF7A0FF034668B9626917705D
S315080053E022681671E288AA4209D220464146FFF78A
S315080053F043FC03460028EBD0042B08BF02231846BB
S31508005400BDE8F0812DE9F04104460E46012998BF12
S3150800541002212BD983699E4228BF022126D2002762
S315080054204FF0010820463146FFF776FA0546C0B127
S31508005430012818D0B0F1FF3F17D0204631463A462A
S31508005440FFF72CFB014688B92369B3F1FF3F1EBF5E
S315080054500133236184F80580A369AB4206D92E4639
S31508005460E0E7002102E0022100E001210846BDE84C
S31508005470F08100BF70B582B0054616461C460B2261
S31508005480FEF798FE052C0BD9B21EE30343EA540433
S3150800549032F8023F13FA84F4A4B25388002BF4D1ED
S315080054A0072204F00F0101F13003392B88BF01F1FF
S315080054B03703013A00A911444B702409F1D1144667
S315080054C07E2102AB134403F8081C62B12B78202B0B
S315080054D00BD0294600230133A34207D011F8010F48
S315080054E02028F8D102E0002300E000232020072A24
S315080054F09FBF02A9891811F8081C013288BF014606
S31508005500E9540133072BF2D902B070BD2DE9F04FEB
S3150800551087B004468769C66903A839460C22FEF790
S3150800552049FE9DF8173013F0010F21D00023FB72B6
S31508005530E3610125384603A932462B46FFF79AFF51
S315080055402046FFF72FFC034620B90135ADB2642D7E
S31508005550F0D1D5E0642D08BF072000F0EF80042BBA
S3150800556018BF184640F0EA809DF81730FB72E661CE
S315080055709DF8173013F0020F08BF012716D033889D
S315080055803BB1002301339BB236F81320002AF9D128
S3150800559000E0002319334EF64F42C4F6C46282FB7C
S315080055A00317DB17C3EBA707BFB2FFE720460021A7
S315080055B0FFF728FA0346002840F0BF800025A846D2
S315080055C0012620682169FEF7A7FE0346002840F059
S315080055D0B48063691B78E52B18BF002B03D101350E
S315080055E0AF4201D18EE0454620463146FFF744FBDF
S315080055F003460028E5D0A0E0E188C9EB0101204672
S3150800560089B2FFF7FFF90346002840F09680A069A3
S31508005610FEF7EAFD01904FF000084FF6FF7549F2D4
S315080056201476C0F60006FF2720682169FEF774FE87
S315080056300346002840F08180D4F81CA061695FFA0F
S3150800564089FB019A4A734FF00F03CB7281F80C80DD
S3150800565081F81A8081F81B800BF1FF3303EB4300B6
S3150800566003EB80000122434602E070462B460132D6
S31508005670AB424ED000F1010E3AF81030B01810F8CF
S31508005680010C0B5408444FEA132C80F801C0002B78
S3150800569049D070460C2AEAD9AB4202D03AF8103003
S315080056A00BB94BF0400B81F800B023684FF00101AD
S315080056B0197120464146FFF7DFFA034600283CD118
S315080056C009F1FF391FFA89F9B9F1000FACD12DE0BC
S315080056D0636903F12001002203F8012B8B42FBD1F9
S315080056E06069A1690B22FEF765FD6369A269D27A32
S315080056F002F018021A73236801221A7100201DE0AD
S3150800570007201BE0013F1FFA87F9B9F1000F0DD0FA
S3150800571072E706EB020E1EF801EC01F80E708E44D5
S315080057208EF80170B6E70C2A9FD9BAE72068216976
S31508005730FEF7F2FD0028CBD000E0184607B0BDE81A
S31508005740F08F00BF88B940F20C63C2F200031B68F1
S315080057500BB100221A7009B100230B7040F20C63DA
S31508005760C2F200031960002070470B20704700BF83
S315080057702DE9F0438FB0019115460446002800F044
S3150800578094800023036001A805A902F01E02FEF713
S31508005790F9FD002840F08B8005F01F0702AB0B933C
S315080057A040F20843C2F200030C9305A80199FFF7DB
S315080057B0CBFB0A9E034600287FD1002E78D17BE0DA
S315080057C05BB1042B40F0858005A8FFF79FFE47F0E4
S315080057D008070A9E034638B17BE0F37A13F0110FE7
S315080057E070D115F0040F6FD117F0080F3CD0FDF7F4
S315080057F0F9FCB073C0F30723F373030C3374000E7C
S3150800580070740025F57235777577B577F577DDF815
S31508005810148040463146FEF7D7FCB576F5763575E1
S315080058207575012388F804300546E8B1D8F8309034
S3150800583040462946FFF7E6FD0346002849D1059864
S31508005840013DC5604946FEF767FD03460AE0F37A5F
S3150800585013F0100F3AD115F0020F05D013F0010F0F
S3150800586036D101E0002B34D117F0080F18BF47F0E6
S315080058702007059D2B6BE3612662A77128463146F2
S31508005880FEF7A2FC2061F27FB37F1B0443EA0263A2
S31508005890327F1343727F43EA0223E3600020A0604D
S315080058A0A0612560EB88A38014E0092012E011E0CE
S315080058B015F01C0F91D1CAE7062315F01C0F7FF4CB
S315080058C07FAFCFE7072304E0082302E0042300E0C4
S315080058D0072318460FB0BDE8F08300BF2DE9F04F47
S315080058E083B004460F4690461E4600233360FEF7F3
S315080058F02DFD002840F0BF80A37913F0800F18BF54
S31508005900022040F0BC8013F0010F08BF072000F00A
S31508005910B680E568A368ED1AA84538BF4546002D48
S3150800592000F0AA8004F124030193A368C3F30802D4
S31508005930002A40F08680206890F802A00AF1FF3A13
S315080059400AEA532A1AF0FF0A17D10BB9206902E0AE
S315080059506169FEF7E1FF012805D8A37963F07F03A3
S31508005960A37102208BE0B0F1FF3F05D1A37963F064
S315080059707F03A371012082E06061D4F8008040466D
S315080059806169FEF7BDFF814628B9A37963F07F03F5
S31508005990A371022073E0D1445FEA552B29D098F809
S315080059A002300BEB0A029A4288BFCAEB030B98F83F
S315080059B0010039464A465FFA8BF3FDF779FB28B1B1
S315080059C0A37963F07F03A371012058E0A37913F04C
S315080059D0400F0BD0A369C9EB0300834506D907EB33
S315080059E0402001994FF40072FEF7E4FB4FEA4B2B77
S315080059F035E0A2694A4522D0A37913F0400F10D0AA
S31508005A0098F8010001990123FDF784FB28B1A379D1
S31508005A1063F07F03A371012031E0A37923F04003EB
S31508005A20A3712368587801994A460123FDF740FB7C
S31508005A3028B1A37963F07F03A37101201FE0C4F89E
S31508005A401890A168C1F30801C1F5007B5D4538BF10
S31508005A50AB462144384624315A46FEF7ABFB5F4431
S31508005A60A3685B44A36033685B443360B5EB0B05FE
S31508005A707FF45BAF02E002E0002000E0002003B004
S31508005A80BDE8F08F2DE9F04F83B004460F46154662
S31508005A901E4600233360FEF759FC002840F0DA80E2
S31508005AA0A37913F0800F18BF022040F0D48013F0BA
S31508005AB0020F08BF072000F0CE80E368DD4280F0C1
S31508005AC0BE80002D00F0BB8004F124030193A36877
S31508005AD0C3F30802002A40F09580206890F802B0C7
S31508005AE00BF1FF3B0BEA532B1BF0FF0B21D13BB904
S31508005AF0236963B90021FFF759F80346206103E0DB
S31508005B006169FFF753F80346002B00F09880012BD4
S31508005B1005D1A37963F07F03A37102209BE0B3F15B
S31508005B20FF3F05D1A37963F07F03A371012092E0BB
S31508005B306361A37913F0400F11D02368587801994F
S31508005B40A2690123FDF7E6FA28B1A37963F07F037A
S31508005B50A37101207FE0A37923F04003A371D4F851
S31508005B60008040466169FEF7CBFE814628B9A379D5
S31508005B7063F07F03A37102206DE0D9445FEA552ADA
S31508005B8029D098F802300AEB0B029A4288BFCBEB71
S31508005B90030A98F8010039464A465FFA8AF3FDF780
S31508005BA0B9FA28B1A37963F07F03A371012052E003
S31508005BB0A369C9EB03018A450AD9019807EB412174
S31508005BC04FF40072FEF7F6FAA37923F04003A371A7
S31508005BD04FEA4A2A28E0A3694B4511D0A268E36830
S31508005BE09A420DD298F8010001994A460123FDF719
S31508005BF05FFA28B1A37963F07F03A37101202AE035
S31508005C00C4F81890A068C0F30800C0F5007A554596
S31508005C1038BFAA462044243039465246FEF7CAFA07
S31508005C20A37943F04003A3715744A3685344A36080
S31508005C30336853443360B5EB0A057FF448AFA3686D
S31508005C40E268934288BFE360A37943F02003A37117
S31508005C50002000E0FFE703B0BDE8F08F38B5044642
S31508005C60FEF774FB002849D1A37913F0200F46D01C
S31508005C7013F0400F0DD0214651F8243B5878A269FD
S31508005C800123FDF747FA00283BD1A37923F0400307
S31508005C90A3712068E169FEF73FFB002833D1256A26
S31508005CA0EB7A43F02003EB72E3682B77A3891B0A90
S31508005CB06B77E389AB77E37BEB772369AB76C3F343
S31508005CC00722EA761B0C2B751B0A6B75FDF78AFAF9
S31508005CD0A875C0F30723EB75030C2B76000E6876C0
S31508005CE00023AB74EB74A37923F02003A371236814
S31508005CF001221A712068FEF7A5FD38BD38BD0020BF
S31508005D0038BD012038BD38BD10B50446FFF7A6FFDB
S31508005D10034608B900222260184610BD70B504462D
S31508005D200D46FEF713FB002840F0BD80A37913F05B
S31508005D30800F40F0B980E268AA4205D203F0020358
S31508005D40DBB2002B08BF1546A2680023A360002D0E
S31508005D5000F0AC802068867876026AB1013A691E3E
S31508005D60B1FBF6F1B2FBF6F3994205D373421A403A
S31508005D70A260AD1A616918E02169A9B9FEF716FF94
S31508005D800146012805D1A37963F07F03A371022098
S31508005D9070BDB0F1FF3F18BF206105D1A37963F04C
S31508005DA07F03A371012070BD6161002940D0B5420F
S31508005DB02BD9A27912F0020F05D02068FEF7F6FE5D
S31508005DC0014620B920E02068FEF7A6FD0146B1F19C
S31508005DD0FF3F05D1A37963F07F03A371012070BD4E
S31508005DE0012903D922689269914205D3A37963F000
S31508005DF07F03A371022070BD6161A2683244A2606C
S31508005E00AD1BAE42D5D300E03546A2682A44A2604F
S31508005E10C5F3080272B12068FEF772FD28B9A379A6
S31508005E2063F07F03A371022070BD00EB552502E0E5
S31508005E30002500E00025A368C3F3080343B3A2695D
S31508005E40AA4225D0A37913F0400F11D0214651F864
S31508005E50243B58780123FDF75DF928B1A37963F04F
S31508005E607F03A371012070BDA37923F04003A371BA
S31508005E70214651F8243B58782A460123FDF718F99C
S31508005E8028B1A37963F07F03A371012070BDA561D2
S31508005E90A368E26893420BD9E360A37943F0200331
S31508005EA0A371002070BD70BD022070BD002070BDBA
S31508005EB0002070BD30B58FB00EAB43F8340D0D46DB
S31508005EC0184605A90022FEF75DFA0446A0B902ABFA
S31508005ED00B9340F20843C2F200030C9305A80199FC
S31508005EE0FFF732F8044638B90A9B23B105A82946B4
S31508005EF0FEF712FC00E0062420460FB030BD00BFB6
S31508005F0030B599B018AB43F85C0D18460FA90122B5
S31508005F10FEF738FA034600284DD103AB159340F235
S31508005F200843C2F2000316930FA80199FFF70CF86D
S31508005F30034600283FD11499062300293BD0CC7A82
S31508005F4014F0010F18BF072335D124E0012D98BF9F
S31508005F50022330D906A80FA92422FEF72BF90895A3
S31508005F6006A80221FEF74EFD034620BB06A800211F
S31508005F70FFF784F90346E8B1042814D01BE02DB1D5
S31508005F800F982946FFF73EFA0346A0B90F98FEF781
S31508005F9059FC03460FE00F98FEF716F9054614F06C
S31508005FA0100FD3D1FFE70FA8FFF700FA0346002822
S31508005FB0E5D000E00723184619B030BD2DE9F043B7
S31508005FC083B081469046054600244E1E012711E0FF
S31508005FD0404601A93A466B46FFF780FC009B012B19
S31508005FE00AD19DF804300D2B04D005F8013B013485
S31508005FF00A2B01D0A642EBDC00232B709C4214BF6F
S315080060004846184603B0BDE8F08300BF30B583B0F4
S3150800601004460D460A2802D10D20FFF7F7FF02A90C
S3150800602001F8084D28466946012201ABFFF72AFD0B
S315080060300198012814BF4FF0FF30012003B030BD8E
S3150800604070B505460E46007860B100243146FFF764
S31508006050DDFFB0F1FF3F08D0013415F8010F002825
S31508006060F4D101E0002070BD204670BD7F2821D9FB
S3150800607041B9C7281EBF49F60412C0F6000201231B
S315080060800AD112E0FF2814D8803849F60413C0F65E
S31508006090000333F81000704732F8021F814205D01A
S315080060A001339BB2802BF7D100E000238033D8B2AE
S315080060B070470020704700BF61280CD049F224724F
S315080060C0C0F600020021013132F8023F53B1834283
S315080060D0F9D10BB97047002149F60423C0F600032D
S315080060E033F81100704700BF30B4013A8D18A94241
S315080060F014D20B461C785A7802EB042292B210444A
S3150800610080B2824284BF013080B202339D42F1D808
S31508006110CB432B4423F0010302331944A94207D188
S315080061200B781B02184480B2834284BF013080B2C8
S3150800613030BC704738B542F62004C2F20004657CCC
S31508006140143D237C05EB0325ADB2284480B204F147
S315080061501A010822FFF7C8FF04F122012A46FFF7B1
S31508006160C3FF034620B1000A40EA032080B238BDC7
S315080061704FF6FF7038BD00BF70B4C4780C44E4B263
S3150800618042F29873C2F20003DC700D0A82782A4440
S31508006190D2B29A7046785E700078187095420DD91A
S315080061A00136F6B242F29873C2F200035E702EB957
S315080061B042F29873C2F2000301301870C9B28C42D9
S315080061C017DA0132D2B242F29873C2F200039A7019
S315080061D07AB942F29873C2F200035A780132D2B2FF
S315080061E05A7032B942F29873C2F200031A78013231
S315080061F01A7070BC704700BF10B5014642F2A4740D
S31508006200C2F2000420680830FFF7B6FF226842F29F
S315080062109873C2F2000319781172597851729978F5
S315080062209172DB78D37210BD08B500200649142296
S31508006230FFF75AFF034620B1000A40EA032080B25E
S3150800624008BD4FF6FF7008BD2E28002008B50620A9
S31508006250FFF770FF08BD00BF42F61003C2F2000345
S3150800626000221A8042F2A873C2F200035A7640F25C
S315080062702463C2F2000301221A7040F21863C2F2C4
S3150800628000034FF480621A80704700BF40F224630F
S31508006290C2F2000300221A7042F61003C2F200038B
S315080062A01B882BB942F61003C2F200031880704708
S315080062B040F22463C2F2000301221A70704700BF3D
S315080062C038B542F2A473C2F200031C6842F2A07306
S315080062D0C2F20003A54A1A6042F29473C2F200039E
S315080062E01A60032813D1637E03F00F03032B40F0D3
S315080062F05B87238A002B40F0578742F29C73C2F2D1
S31508006300000308221A7001F07BFB00F097BD0228F3
S3150800631040F09E8040F21463C2F20003DA7801323C
S31508006320D2B2DA70C2B940F21463C2F200039A78A4
S315080063300132D2B29A707AB940F21463C2F20003FB
S315080063405A780132D2B25A7032B940F21463C2F2A4
S3150800635000031A7801321A7042F29073C2F20003EF
S3150800636000221A8042F66263C2F200031A80637E34
S3150800637003F0FD02052A09D1A37E0133DBB2A37619
S31508006380782B04BF0023637600F00EBF002B00F0C5
S315080063900B87228A002A4CD0A27E511EA176002A9B
S315080063A040F00287E27E082A05D0591EC9B20129A3
S315080063B014D8052A12D10023637642F29C73C2F2DE
S315080063C0000380221A7001F01BFB42F62003C2F27A
S315080063D00003142283F82F2000F063BE042A9DBF11
S315080063E003219140C9B23021A1760132E27603F049
S315080063F00F03013B072B00F2D786DFE813F05D0297
S3150800640008001000AC04D506AC04D506AC0442F668
S315080064102003C2F20003002283F82F2053E242F23F
S315080064209C73C2F2000304221A7001F0E9FA00F024
S3150800643056BD03F00F03032B40F0B68642F29C7359
S31508006440C2F2000308221A7001F0DAFA00F0F6BC6C
S3150800645042F62003C2F200039B7B452B40F0A4863C
S3150800646042F62003C2F20003197C5A7C02EB012093
S3150800647042F29073C2F200031B88984200F3948696
S3150800648084B242F29073C2F200031C8042F62003E3
S31508006490C2F200031B7D13F03F0F40F0858642F6DB
S315080064A02003C2F200035B7D002B40F07D8642F696
S315080064B01C03C2F200031D882DB942F61C03C2F262
S315080064C000035B88A3B142F62003C2F20003DB8B0C
S315080064D0AB4240F0698642F62002C2F2000242F65A
S315080064E01C03C2F20003128C5B889A4240F05C8659
S315080064F0FFF79AFE4FF6FF73984240F0558642F62C
S315080065002003C2F20003DB7D062B31D0012B40F0BD
S315080065104B8642F62003C2F2000393F82230082B7A
S3150800652040F0428642F62003C2F20003002283F8B6
S3150800653022209A8C4FF6F6739A4242F62003C2F24C
S3150800654000038CBF093208329A8442F62003C2F24D
S3150800655000035A8BDA839A8B1A845D8342F61C02EF
S31508006560C2F2000252889A8300F017BE562800200D
S31508006570FFF76CFE4FF6FF73984240F0158642F21D
S31508006580A873C2F20003597E81B342F62002C2F212
S31508006590000242F2A873C2F20003928C9B889A42C8
S315080065A024D142F62002C2F2000242F2A873C2F2D5
S315080065B00003528CDB889A4218D142F62002C2F2B6
S315080065C0000242F2A873C2F20003528B1B889A4259
S315080065D00CD142F62002C2F2000242F2A873C2F2BD
S315080065E00003928B5B889A4200F08D8142F6200365
S315080065F0C2F2000393F82F3003F03F03022B1CD19D
S3150800660042F62003C2F200039A8C40F21063C2F2EB
S3150800661000031A8040F22463C2F2000300211970B5
S3150800662042F61003C2F200031B8893427BD040F265
S315080066302463C2F2000301221A7042F62003C2F252
S31508006640000393F82F3013F0040F40F0AD8542F69F
S315080066502003C2F20003142283F82F2042F290721C
S31508006660C2F2000228211180502283F82E2093F8C6
S31508006670295093F82D2083F8292093F8284093F879
S315080066802C2083F8282083F82C4093F8270093F8C9
S315080066902B2083F8272083F82B0093F8262040F236
S315080066A02461C2F200010A7093F82A1083F82610B2
S315080066B083F82A20691CC9B283F82D10C1B9611C58
S315080066C0C9B242F62003C2F2000383F82C1079B946
S315080066D0411CC9B242F62003C2F2000383F82B100C
S315080066E031B942F62003C2F20003013283F82A20A8
S315080066F042F62003C2F20003598C40F21062C2F23D
S31508006700000211809A8C5A8499845A8BDA839A8B60
S315080067101A8442F61C02C2F2000211885983528872
S315080067209A8300F00DBD42F2A873C2F200035B7EA5
S3150800673023B1072B40F04C8500F042BD42F2A4710C
S31508006740C2F2000142F2A873C2F200030B600321F1
S3150800675099761976002199750420D875D9769A8084
S3150800676042F62004C2F20004628CDA80628B1A8038
S31508006770A28B5A800120587640F21462C2F20002B7
S31508006780117819735178597391789973D278DA73A5
S31508006790188294F82920DA7294F828209A7294F8C4
S315080067A027205A7294F826201A72FFF725FD94F8C6
S315080067B02E3003F0F002502A7ADD1B095C1FA40074
S315080067C040F22563C2F200031A78002342F620013C
S315080067D0C2F200015AE0CA1892F8362072B940F29D
S315080067E02461C2F200010B7040F22563C2F2000375
S315080067F01A7042F2A874C2F200045DE0012A02D1BE
S315080068000133DBB242E0022A2BD10D1895F8375036
S31508006810042D26D140F22462C2F20002137040F21F
S315080068202563C2F2000302221A7042F62003C2F25E
S315080068300003034493F8382093F8393043EA0222D8
S3150800684040F21063C2F200031A8040F20A639A42C9
S3150800685038BF134642F2A874C2F200046382A382C8
S315080068602AE0084490F8370070B940F22461C2F271
S3150800687000010B7040F22563C2F200031A7042F25F
S31508006880A874C2F2000417E00344DBB21846A34218
S31508006890A1DB40F22461C2F200010B7040F22563CD
S315080068A0C2F200031A7042F2A874C2F2000403E0AE
S315080068B042F2A874C2F2000442F62003C2F20003B0
S315080068C0102283F82F2042F62003C2F2000393F821
S315080068D02F2042F0020283F82F20022283F8362066
S315080068E0042283F83720062283F838200A2283F800
S315080068F0392042F29072C2F200022C2111806022E5
S3150800690083F82E20DAE342F2A473C2F2000342F2BD
S31508006910A872C2F200021A6042F29C73C2F2000325
S3150800692000221A7042F62003C2F2000393F82F30B1
S3150800693013F0040F0ED042F2A873C2F200035A767F
S3150800694042F29C73C2F2000320221A7001F058F832
S3150800695000F02ABC42F62002C2F2000292F82E008B
S315080069600009800040F22462C2F200021070143C52
S31508006970201A80B242F29072C2F20002108001F030
S315080069800F01022903D103F03F02122A1DD010B9C4
S3150800699013F0030F19D042F62001C2F2000142F2A9
S315080069A0A872C2F20002C98C1289914240F06E8325
S315080069B042F62001C2F2000142F2A872C2F20002B7
S315080069C0098D5289914240F0618313F0100F77D0F8
S315080069D042F2A873C2F20003198A002970D003F1A3
S315080069E00C00FFF7C9FB42F62003C2F2000393F836
S315080069F02A4042F29873C2F200031B78A3425FD181
S31508006A0042F62003C2F2000393F82B0042F2987371
S31508006A10C2F200035B78834252D142F62003C2F2E7
S31508006A20000393F82C1042F29873C2F200039B7885
S31508006A308B4245D142F62003C2F2000393F82D207B
S31508006A4042F29873C2F20003DB78934238D142F2DD
S31508006A50A873C2F200031C7358739973DA73DB7E4A
S31508006A6003BB42F2A873C2F20003987D197E9A7E90
S31508006A70891AA1EBD001C9B2CAB20844C0B2987546
S31508006A8012F0800F1CBF4A42D2B242F2A873C2F279
S31508006A900003D97DA1EB91010A44D2B2DA7502EB63
S31508006AA0D0021A7642F29C73C2F2000301221A70CF
S31508006AB042F2A873C2F200031A7E9A7600221A825C
S31508006AC042F2A873C2F200035A7E02F00F03013B9A
S31508006AD0072B00F26983DFE813F008003A00040187
S31508006AE051029B02C702D902390242F29C73C2F2D2
S31508006AF000031B7813F0010F00F0568342F2A873C7
S31508006B00C2F2000303225A7642F29C72C2F20002D3
S31508006B104021117000221A8242F29073C2F20003D9
S31508006B20188838B142F29C73C2F2000342221A70E6
S31508006B30FFF762FB42F66263C2F2000300221A8084
S31508006B4000F05EFF42F2A874C2F2000476E142F257
S31508006B509C73C2F200031B7813F0010F00F0B1809A
S31508006B6042F62003C2F2000393F82F3003F03F03E6
S31508006B70122B40F0A68042F62003C2F2000393F8D7
S31508006B802E3003F0F002502A6DDD1B095C1FA400AD
S31508006B9040F22563C2F200031A78002342F6200168
S31508006BA0C2F2000152E0CA1892F8362052B940F2F1
S31508006BB02461C2F200010B7040F22563C2F20003A1
S31508006BC01A7050E0012A02D10133DBB23EE0022AF4
S31508006BD02BD10D1895F83750042D26D140F2246292
S31508006BE0C2F20002137040F22563C2F200030222C9
S31508006BF01A7042F62003C2F20003034493F83820C1
S31508006C0093F8393043EA022240F21063C2F20003D5
S31508006C101A8040F20A639A4228BF1A4642F2A873BB
S31508006C20C2F200035A829A821DE0084490F837009F
S31508006C3050B940F22461C2F200010B7040F225639C
S31508006C40C2F200031A700EE00344DBB21846A342F0
S31508006C50A9DB40F22461C2F200010B7040F2256301
S31508006C60C2F200031A7042F2A874C2F200040323A7
S31508006C70637642F62003C2F2000393F826202272B6
S31508006C8093F82720627293F82820A27293F8293085
S31508006C90E3720120FFF7B0FA42F29C73C2F20003D6
S31508006CA042221A700022228242F29073C2F2000334
S31508006CB01A8042F66263C2F200031A8000F0A0FE50
S31508006CC0BCE042F29C73C2F2000320221A7000F064
S31508006CD097FE42F2A473C2F200031B6800225A769A
S31508006CE0ABE442F62003C2F2000393F82F3013F008
S31508006CF0010F38D012F0100F35D142F2A873C2F244
S31508006D0000031B8A002B40F04F8242F29074C2F2B5
S31508006D1000042088013080B2FFF76EFA42F29C73B5
S31508006D20C2F200031A7842F010011970238833B1B1
S31508006D3042F29C73C2F2000342F012021A7000F08B
S31508006D405FFE42F2A874C2F20004012323820823DC
S31508006D5063760023E37642F62003C2F2000311228B
S31508006D6083F82F209DE113F0200F18D042F6200358
S31508006D70C2F2000393F83400000293F8351042F289
S31508006D80A073C2F2000340EA01051C682C441C608B
S31508006D9042F29073C2F200031888411B198042F22E
S31508006DA09073C2F20003188860B112F0100F09D16F
S31508006DB042F29C73C2F200031A7842F002021A7079
S31508006DC0FFF71AFA42F62003C2F2000393F83020BE
S31508006DD093F8313003EB02239BB240F21062C2F201
S31508006DE00002138042F2A872C2F20002928A93420B
S31508006DF000D823B940F21063C2F200031A8042F2A7
S31508006E00A873C2F2000340F21062C2F200021288AE
S31508006E105A8242F29C73C2F200031B7813F0030FE6
S31508006E2000F0C28142F66263C2F2000300221A80B1
S31508006E3000F0E6FD42F2A874C2F2000442F29C7326
S31508006E40C2F200031B7813F0200F0ED042F66263DD
S31508006E50C2F2000300221A80627642F62003C2F2CA
S31508006E600003142283F82F201BE113F0100F12D011
S31508006E7042F66263C2F2000300221A8001232382CB
S31508006E8004236376E27642F62003C2F20003112257
S31508006E9083F82F2005E142F66262C2F200021288E8
S31508006EA0DAB113F0010F1CBF0023238201D1218A16
S31508006EB071B9618A8A4282BF42F66263C2F20003EE
S31508006EC0198042F66263C2F200031B88238204E03B
S31508006ED042F66263C2F2000319800023E37642F2A7
S31508006EE0A073C2F2000342F29472C2F20002126860
S31508006EF01A6042F66263C2F200031B887BB1238ADA
S31508006F006BB142F29072C2F200022833138042F645
S31508006F102003C2F20003182283F82F20C7E042F2AA
S31508006F209C73C2F200031B7813F0020F00F03C8139
S31508006F3042F29073C2F2000328221A8042F6200316
S31508006F40C2F20003102283F82F20B0E042F29C73AD
S31508006F50C2F200031B7813F0010F00F0258142F2FC
S31508006F60A873C2F2000300225A7642F29C73C2F258
S31508006F70000310221A7000F043FD15E142F29073E7
S31508006F80C2F20003188808B1FFF736F942F6200363
S31508006F90C2F2000393F82F3013F0010F1FD042F20C
S31508006FA09C73C2F200031B7813F0010F42F2A87318
S31508006FB0C2F200031FBF07225A7600229A7612BF32
S31508006FC01A8206225A760120FFF716F942F29C73B6
S31508006FD0C2F2000310221A7000F012FD56E042F2C7
S31508006FE09C73C2F200031B7813F0010F08D042F21B
S31508006FF0A873C2F2000305225A7600221A82D3E049
S3150800700042F29073C2F200031B88002B3ED1CBE0FC
S3150800701042F29073C2F20003188808B1FFF7ECF841
S3150800702042F62003C2F2000393F82F3013F0010F43
S3150800703013D042F2A873C2F2000307225A7600223E
S315080070409A760120FFF7D8F842F29C73C2F2000341
S3150800705010221A7000F0D4FC18E042F29073C2F2C3
S3150800706000031B8893B99FE042F29C73C2F20003A7
S315080070701B7813F0010F00F0978042F2A873C2F252
S31508007080000307225A7600229A768DE042F62003FC
S31508007090C2F20003102283F82F2042F2A874C2F22B
S315080070A0000442F29073C2F2000328221A8042F6C4
S315080070B02003C2F20003502283F82E20227A42F6D9
S315080070C02003C2F2000383F82A20627A83F82B2071
S315080070D0A27A83F82C20E27A83F82D20227B83F883
S315080070E02620627B83F82720A27B83F82820E27B70
S315080070F083F829200622DA75A2885A84E2889A84B7
S3150800710042F61C02C2F200021188598352889A83F9
S315080071102288DA8362881A84637E13F0100F42F697
S315080071202003C2F200031DBF002283F8312083F832
S315080071303020062202BF83F830200A2283F8312045
S3150800714042F62004C2F200044023A37542F290736B
S31508007150C2F200031B881A0A22746374002584F895
S31508007160355084F834506586FFF770F8C04360865A
S315080071704523A373E5736575257540F21263C2F25C
S3150800718000031A88013292B21A80130AA374E274B1
S315080071902583FFF749F8C043208342F29C73C2F265
S315080071A0000300221A7038BD42F29073C2F200033F
S315080071B000221A8042F29C73C2F200031A7038BD8C
S315080071C040F22463C2F2000301211970FFF7B6BA30
S315080071D040F22463C2F2000301221A70E4E700BFFA
S315080071E0030A43EA002080B2704700BF10B5044680
S315080071F00A1E0FDD42F66263C2F200031A8042F2EB
S315080072009473C2F200031868844203D0214692B2EE
S3150800721002F046F910BD00BF2DE9F00340F22663DF
S31508007220C2F200034FF0000C83F800C040F2286554
S31508007230C2F200052B4601221F461C88CCB15E8887
S31508007240BEB1B0F80080A04513D14488B44210D12D
S3150800725040F22663C2F2000383F800C0086878602B
S315080072608B883B8140F28963C2F200031B78BB72AC
S315080072705AE0541CE4B20C33092C02D09446224638
S31508007280DAE72B4600221E461C884CB95C883CB9B6
S3150800729040F22663C2F200031A70082A36D104E0C7
S315080072A00132D2B20C33082AEDD1002340F28962AA
S315080072B0C2F200021678B0461F4699465FFA83FC6A
S315080072C0AA7AC2EB0804BC42C2BFC2EB0602E14678
S315080072D0D7B201330C35082BF0D140F22763C2F23E
S315080072E000031F7040F28863C2F2000383F800901F
S315080072F040F22663C2F2000383F8009040F2286346
S31508007300C2F2000309EB490903EB89060268334612
S3150800731043F8042B0A6872608A889A8040F2896367
S31508007320C2F200031B78B372BDE8F003704700BFD2
S31508007330F0B440F28963C2F200031E780136F6B251
S315080073401E7040F22863C2F200030122002740F2B1
S315080073502664C2F2000458881988014389B259B1D3
S31508007360997A711A772907DD194601F8017B5F704A
S31508007370013101F8017B0F7022700132D2B20C3351
S31508007380092AE8D1F0BC704738B542F29073C2F2C8
S3150800739000031B88292B06D842F29073C2F2000319
S315080073A000221A8038BD42F29073C2F2000300220E
S315080073B01A8042F62003C2F200039B8AB3F5807F47
S315080073C003D0B3F5007F59D038BD42F62002C2F289
S315080073D0000242F61C03C2F20003D28C1B889A42B2
S315080073E069D142F62002C2F2000242F61C03C2F23A
S315080073F00003128D5B889A425DD12F4CA51F20464B
S315080074002946FFF709FFA4F11C03002204F8082CFB
S31508007410022204F8072C54F8062C626034F8022C71
S31508007420228140F21C62C2F20002106844F8060C7F
S31508007430928824F8022C44F8160C24F8122C626858
S3150800744044F81C2C228924F8182C9A8B62816288AD
S31508007450A28142F61C02C2F2000211889983528860
S315080074606280082204F8102C062204F80F2C42F237
S315080074709073C2F200032A221A8038BD42F620020F
S31508007480C2F2000242F61C03C2F20003D28C1B8829
S315080074909A4210D142F62002C2F2000242F61C03BA
S315080074A0C2F20003128D5B889A4204D1024908464B
S315080074B00639FFF7B1FE38BD3C28002038B542F63C
S315080074C02003C2F20003D98B8AB24FF6FF739A42A1
S315080074D015D142F62003C2F20003188C4FF6FF734B
S315080074E098420CD142F62003C2F2000349F6E43270
S315080074F0C0F600021068186092889A80ADE042F6DD
S315080075001C03C2F200031B885A4042F61803C2F253
S3150800751000031B881A4212D142F62003C2F2000366
S315080075201A8C90B242F61C03C2F200035B885840DC
S3150800753042F61803C2F200035B8818420CD040F2E8
S315080075408C63C2F2000342F61402C2F200021188EA
S31508007550198052885A8005E040F28C63C2F2000313
S3150800756019805A8040F28C63C2F2000318885D883D
S3150800757040F22863C2F2000300221C4619888142A1
S315080075800AD15988A94207D140F22663C2F20003FC
S315080075901A70082A58D109E00132D2B20C33082AE7
S315080075A0EBD140F22663C2F200031A7042F62004B9
S315080075B0C2F200042046FF21062201F0C5FF00237F
S315080075C084F8203084F8213084F8223084F8233077
S315080075D084F8243084F8253040F21C62C2F2000296
S315080075E01168C4F8061092886281C4F8161062837E
S315080075F040F28C62C2F200021188E1845288228528
S3150800760042F61C02C2F200021188A1835288E28364
S31508007610237501226275A373E273082222746374C8
S315080076200623A3740423E37422730623637342F2C6
S31508007630A073C2F2000336341C6042F29073C2F2A1
S3150800764000032A221A8038BD42F62003C2F200033C
S3150800765054F8040F1860A2889A8042F62003C2F2F2
S31508007660000340F21C62C2F200021168C3F8061059
S3150800767092885A8108221A7300225A7342F290732A
S31508007680C2F200031A880E321A8038BD08B500F017
S3150800769017FC01F093FE01F077FE00F095FC00F070
S315080076A00FF800F0FBFB08BD08B500F00BFC01F075
S315080076B0A1FE00F0C7FD00F01BF800F0C7FB08BDEF
S315080076C010B500F0E1F901F00BF840F2E404C2F25B
S315080076D000040123237001F08DFB0023237001F0C1
S315080076E0ABFC0223237000F0A9F80323237010BD16
S315080076F008B540F29060C2F2000001F0F9F80128DE
S315080077000BD140F2E403C2F2000301221A7040F2E0
S315080077109060C2F2000000F0D7F940F29060C2F221
S31508007720000001F0BBFB01280BD140F2E403C2F2D2
S31508007730000300221A7040F29060C2F2000000F0C6
S31508007740C3F940F29060C2F2000001F02BFD012857
S315080077500BD140F2E403C2F2000302221A7040F28F
S315080077609060C2F2000000F0AFF940F29060C2F2F9
S31508007770000000F0BFF801280BD140F2E403C2F282
S31508007780000303221A7040F29060C2F2000000F073
S315080077909BF908BD08B501F0BBFC08BD38B5054620
S315080077A00C4640F2E403C2F200031B78012B02D117
S315080077B0C9B201F049F840F2E403C2F200031B78AB
S315080077C01BB92846E1B201F035FB40F2E403C2F2E8
S315080077D000031B78022B03D12846E1B201F0A4FC72
S315080077E040F2E403C2F200031B78032B03D12846B8
S315080077F0E1B200F05DF800F05FF938BD40F2E4034D
S31508007800C2F200031878012804D002280CBF3F20D2
S31508007810402070470820704740F2E403C2F2000394
S315080078201878012804D002280CBF3F204020704752
S315080078300820704708B500F035F908BD08B5FBF70C
S3150800784079FF01F0E9FD40F2D463C2F2000300F5C6
S31508007850FA70186001F0E0FD40F2D063C2F200034E
S3150800786000F51C5010301860FEF7F6FC42F61C03B3
S31508007870C2F200034FF6A9621A8043F613715980C3
S3150800788042F61803C2F200034FF6FF711980002171
S31508007890598042F61403C2F200031A8040F213120A
S315080078A05A804EF60300FEF7F1FCFCF757F808BDC0
S315080078B0F8B542F2A473C2F200031F68FB693B6283
S315080078C08E4659B14E1EB6B20136002307F11C0585
S315080078D0C45CEA1814720133B342F9D10EF10401FB
S315080078E0A7F8641007F12000FFF780FCFB69013355
S315080078F0FB61F8BD10B5FCF743F800283ED042F20C
S315080079009072C2F20002108042F62003C2F200030F
S315080079109C894FF40060FFF763FC844213D1012071
S31508007920FEF7CEFC42F29073C2F200031B882BB31B
S31508007930FFF7C4FDFCF74CF842F29073C2F200035D
S3150800794000221A801AE042F62003C2F200039C893C
S3150800795040F60600FFF744FC84420FD1FFF714FDFA
S3150800796042F29073C2F200031B883BB1FCF730F871
S3150800797042F29073C2F2000300221A8001F04CFD15
S3150800798040F2D463C2F200031B68984222D340F245
S31508007990D462C2F2000203F5FA73136042F2A473CA
S315080079A0C2F2000342F2A872C2F200021A60022072
S315080079B0FEF786FC42F29073C2F200031B884BB1B5
S315080079C0FFF77CFDFCF704F842F29073C2F200035D
S315080079D000221A8001F020FD40F2D063C2F20003B3
S315080079E01B68984209D340F2D062C2F2000203F53E
S315080079F01C5310331360FFF79BFC002010BD00BF1B
S31508007A0010B542F2A473C2F200031C6842F29C73DA
S31508007A10C2F200031B7813F0400F05D00123E3617F
S31508007A200023A4F8643010BD13F0010F1CBF002218
S31508007A30A4F8642013F0040F06D0B4F8641019B142
S31508007A4004F12000FFF7D2FB42F29C73C2F2000356
S31508007A501B7813F0020F0AD00023A4F8643042F210
S31508007A60A073C2F200031868043000F02DF810BDA8
S31508007A7040F2D863C2F20003FE22DA7018710222BD
S31508007A80A3F84420704700BF40F2D863C2F200034F
S31508007A9000221A709A6483F84320A3F844209A7047
S31508007AA05A70704740F2D863C2F200031878003063
S31508007AB018BF0120704700BF40F2D863C2F2000326
S31508007AC0002283F84320704738B504460178FF2919
S31508007AD023D100F08FFA18B91020FFF7C9FF96E1F5
S31508007AE040F2D864C2F200040023637001252570B1
S31508007AF0FF22E270102222716371FFF77FFEA071E8
S31508007B00FFF78AFEE071FFF787FE000A20726572AA
S31508007B10A5720823A4F8443079E140F2D863C2F28A
S31508007B2000031B78012B40F09081C939352900F2F2
S31508007B306B81DFE811F0DB00690169016501690104
S31508007B4069015901FC0042012F01690169016901B6
S31508007B5069016901690169016901690169016901C7
S31508007B6069016901690169016901690169016901B7
S31508007B7069016901690169016901690169016901A7
S31508007B80690169016901690169017F0054003600CC
S31508007B907300690169016901A1006901B900BD00A5
S31508007BA0CE004578FFF72AFE0138854203DD2220FC
S31508007BB0FFF75EFF2BE140F2D865C2F20005281DEB
S31508007BC0A96C627800F0F4FEFF23EB706278AB6C68
S31508007BD01344AB6463780133A5F8443017E145785C
S31508007BE0FFF70CFE0138854203DD2220FFF740FF30
S31508007BF00DE1616840F2D865C2F20005A964281D46
S31508007C00627800F0D5FEFF23EB706278AB6C134404
S31508007C10AB6463780133A5F84430F8E040F2D863E2
S31508007C20C2F20003FF22DA7042689A640122A3F8BE
S31508007C304420ECE040F2D863C2F20003FF22DA7077
S31508007C409B6C406840B11844002213F8011B0A4493
S31508007C50D2B28342F9D100E0002240F2D863C2F2E0
S31508007C600003C3F8072001221A7100225A719A717B
S31508007C700822A3F84420CAE040F2D863C2F20003FF
S31508007C80FF22DA7049F6EC32C0F600029A64002246
S31508007C901A715A719A710721D9711A725A729A729F
S31508007CA00822A3F84420B2E00020FFF7E1FEAEE088
S31508007CB040F2D863C2F20003FF22DA7000221A717A
S31508007CC0597859719A71DA711A720622A3F8442002
S31508007CD09DE040F2D863C2F2000300221A705A707F
S31508007CE0FF22DA700122A3F8442090E040F2D8631C
S31508007CF0C2F200039D6CFFF781FD411E2846621CF7
S31508007D0001F046FB18B93120FFF7B2FE7FE040F2DA
S31508007D10D864C2F20004FF23E370A56CFFF76EFD7A
S31508007D20013D2844A0640123A4F844306FE0457857
S31508007D30FFF764FD0238854203DD2220FFF798FE2F
S31508007D4065E040F2D863C2F20003FF22DA7001222E
S31508007D50A3F84420617839B901F026FB002856D1EA
S31508007D603120FFF785FE52E040F2D863C2F20003E5
S31508007D70986CA21C01F00CFB18B93120FFF778FEAD
S31508007D8045E040F2D863C2F2000361789A6C0A446F
S31508007D909A643CE040F2D864C2F20004FF23E37020
S31508007DA0002525716571FFF729FDA071E57125721A
S31508007DB065720723A4F8443029E040F2D863C2F27A
S31508007DC00003986C616801F0E7FA18B93120FFF7EB
S31508007DD04FFE1CE040F2D863C2F20003FF22DA70BD
S31508007DE00122A3F8442012E000F0C6FD40F2D86351
S31508007DF0C2F20003FF22DA700122A3F8442006E04B
S31508007E003120FFF735FE02E02020FFF731FE40F271
S31508007E10D863C2F2000393F84330012B02D1102035
S31508007E20FFF726FE40F2D863C2F20003B3F8441007
S31508007E300BB2002B09DD40F2D860C2F20000012324
S31508007E4080F843300330FFF7A9FC38BD08B5FFF7C3
S31508007E50F1FC012820D000F0CDF8E8B140F22473F7
S31508007E60C2F200031B78012B16D101F0D5FA40F2B5
S31508007E702873C2F200031B6803F51C53103398429B
S31508007E800AD340F22473C2F2000300221A7000F0EB
S31508007E90BBF808B900F070FD08BD00BF08B540F290
S31508007EA02473C2F2000301221A7001F0B5FA40F2F7
S31508007EB02873C2F200031860FFF7C8FF08BD00BFA9
S31508007EC0704700BF704700BF00F00F03092802D9AA
S31508007ED003F13700704703F1300040F2E803C2F2BD
S31508007EE000031B6803445B7803F00303022B08BFF7
S31508007EF02038C0B2704700BF38B505460C460009A1
S31508007F00FFF7E2FF207005F00F00FFF7DDFF607056
S31508007F100023A370204638BD30B4024603464CF60B
S31508007F20CD40CCF6CC400131A0FB0343DB08FAD1A7
S31508007F30002301F801394CF6CD45CCF6CC45084668
S31508007F40A5FB0243DB0803EB8304A2EB44023032B1
S31508007F5001F801291A46002BF1D130BC704700BF41
S31508007F60F0B440F2E803C2F200031F6800231C467F
S31508007F70C15C7A18527802F00302022A08BF203937
S31508007F80C9B2A1F13002D2B2A1F13A05EDB2162A70
S31508007F9094BF00260126062D8CBF354646F00105FE
S31508007FA065B9092A84BFA1F13702D2B22401E4B225
S31508007FB02244D4B20133022BDAD101E0002000E0DA
S31508007FC02046F0BC704700BF08B540F26C73C2F299
S31508007FD000030020187040F27871C2F20001FDF724
S31508007FE0B1FB30B149F6F430C0F600007C2100F050
S31508007FF069FB08BD40F26C73C2F200031878D0F131
S31508008000010038BF0020704708B5FFF713FC0128A8
S315080080100FD040F26C73C2F200031B785BB9F8F715
S31508008020C5F8012809D140F26C73C2F20003187032
S3150800803008BD002008BD002008BD002008BD00BFFF
S31508008040027840F2E803C2F200031B6899184978DF
S3150800805001F00301022908BF203A532A0ED14078BD
S3150800806003445B7813F0040F0AD031280AD032286B
S315080080700AD0332814BF0320022070470320704714
S3150800808003207047002070470120704770B50446EA
S315080080900230FFF765FF0646054604342046FFF71B
S315080080A05FFF3044C6B2013DADB20234012DF5D8AA
S315080080B02046FFF755FFF643F6B2864214BF002066
S315080080C0012070BD2DE9F04115460F4604460029EA
S315080080D018BF002807D149F6F430C0F6000040F270
S315080080E0362100F0EFFA2046FFF7AAFF06460328D6
S315080080F008BF002000F0A2802046FFF7C7FF00282F
S3150800810000F08C80012E29D016B1022E53D088E0BB
S31508008110A01CFFF725FF8046201DFFF721FF06025A
S315080081203E60A01DFFF71CFF3044386004F10806C6
S31508008130A8F103081FFA88F84046002D7ED00FFAEA
S3150800814088F7002F6FDD00243046FFF709FF285512
S3150800815002360134A4B2BC42F6DB66E0A01CFFF787
S31508008160FFFE8046201DFFF7FBFE06043E60A01DAD
S31508008170FFF7F6FE06EB00263E6004F10800FFF75F
S31508008180EFFE3044386004F10A06A8F104081FFA25
S3150800819088F84046002D51D00FFA88F7002F46DDA3
S315080081A000243046FFF7DCFE285502360134A4B217
S315080081B0BC42F6DB3DE0A01CFFF7D2FE8046201D40
S315080081C0FFF7CEFE06063E60A01DFFF7C9FE06EBCA
S315080081D000463E6004F10800FFF7C2FE06EB0026E3
S315080081E03E6004F10A00FFF7BBFE3044386004F134
S315080081F00C06A8F105081FFA88F84046F5B10FFAEB
S3150800820088F7002F17DD00243046FFF7A9FE28550A
S3150800821002360134A4B2BC42F6DB0EE04FF6FF701C
S315080082200CE000200AE0404608E0404606E04046EA
S3150800823004E0404602E0404600E0404600B2BDE8A1
S31508008240F08100BF70B540F26C73C2F200031B7870
S31508008250002B00F03382012B3FD1F7F7CFFF49F609
S315080082600C40C0F60000F8F713F849F63040C0F69F
S315080082700000F8F70DF8F7F7BBFF0146BD480122E5
S31508008280FDF776FA48B149F65840C0F60000F7F708
S31508008290FFFF0120F7F7ECFF70BD49F66040C0F616
S315080082A00000F7F7F5FF49F66840C0F60000F7F753
S315080082B0EFFF49F68C40C0F60000F7F7E9FF40F2F9
S315080082C07073C2F2000300221A605A6040F26C739F
S315080082D0C2F2000302221A7070BD022B40F0FD8024
S315080082E040F27874C2F2000440F6D030C2F20000C0
S315080082F04FF4807104F50D72FDF760FE94F93A3279
S31508008300002B13DA49F65840C0F60000F7F7C0FF0D
S315080083100220F7F7ADFF04F50D70FDF7F5FC40F206
S315080083206C73C2F2000300221A7070BD00B340F6E7
S31508008330D031C2F20001084601F5C0710022FFF7EC
S31508008340C1FE0546B0F1FF3F12D149F65840C0F6C6
S315080083500000F7F79DFF0320F7F78AFF8548FDF72A
S31508008360D3FC40F26C73C2F2000300221A7070BD8F
S315080083702BB2002B2CDD40F27073C2F200035B684F
S315080083806BB940F27073C2F2000340F6D032C2F203
S315080083900002D2F880211A602DB25D6018E040F61E
S315080083A0D032C2F20002D2F8801140F27072C2F2E4
S315080083B00002126891423EBF40F27072C2F2000299
S315080083C0116040F27072C2F2000203FA85F353603C
S315080083D040F27873C2F20003D3F83C22D3F8403255
S315080083E09A4240F06B8163480021FDF797FC90B1F3
S315080083F049F65840C0F60000F7F74AFF0420F7F799
S3150800840037FF5C48FDF780FC40F26C73C2F200034C
S3150800841000221A7070BD49F66040C0F60000F7F7F2
S3150800842037FF49F6BC40C0F60000F7F731FF40F2C7
S315080084307075C2F2000540F22C74C2F20004686836
S315080084402146FFF769FD2046F7F722FF49F6C8409F
S31508008450C0F60000F7F71CFF2E68300E2146FFF71E
S315080084604BFDC6F30740A11CFFF746FDC6F30720E0
S31508008470211DFFF741FDF0B2A11DFFF73DFD204686
S31508008480F7F706FF49F66C50C0F60000F7F700FF4D
S315080084902868696800F080FF90B949F65840C0F628
S315080084A00000F7F7F5FE0520F7F7E2FE3148FDF77D
S315080084B02BFC40F26C73C2F2000300221A7070BDE6
S315080084C049F66040C0F60000F7F7E2FE40F26C732A
S315080084D0C2F2000303221A7070BD032B40F0EE802F
S315080084E040F27874C2F2000440F6D030C2F20000BE
S315080084F04FF4807104F50D72FDF760FD94F93A3278
S31508008500002B13DA49F6E440C0F60000F7F7C0FE80
S315080085100220F7F7ADFE04F50D70FDF7F5FB40F206
S315080085206C73C2F2000300221A7070BD20B340F6C5
S31508008530D032C2F20002104602F5C07102F580720E
S31508008540FFF7C0FD0546B0F1FF3F15D149F60850C3
S31508008550C0F60000F7F79CFE0320F7F789FE0548EA
S31508008560FDF7D2FB40F26C73C2F2000300221A70C8
S3150800857070BD00BFAC0900202BB2002B59DD49F6AF
S315080085802C50C0F60000F7F783FE2DB240F22C748B
S31508008590C2F2000428462146FFF7BEFC2046F7F73C
S315080085A077FE49F63C50C0F60000F7F771FE40F634
S315080085B0D036C2F2000696F883012146FFF79CFCE6
S315080085C096F88201A11CFFF797FC96F88101211DF8
S315080085D0FFF792FC96F88001A11DFFF78DFC204657
S315080085E0F7F756FE49F66C50C0F60000F7F750FE4E
S315080085F0D6F88001294606F5807200F0C9FE90B9C2
S3150800860049F65840C0F60000F7F742FE0620F7F78D
S315080086102FFE2B48FDF778FB40F26C73C2F200037D
S3150800862000221A7070BD49F66040C0F60000F7F7E0
S315080086302FFE40F27873C2F20003D3F83C22D3F837
S3150800864040329A423AD149F65450C0F60000F7F73C
S315080086501FFE00F0A9FE90B949F65840C0F6000082
S31508008660F7F716FE0720F7F703FE1548FDF74CFB4C
S3150800867040F26C73C2F2000300221A7070BD49F60C
S315080086806040C0F60000F7F703FE49F67050C0F6E2
S315080086900000F7F7FDFD0A48FDF736FB49F6885056
S315080086A0C0F60000F7F7F4FD40F26C73C2F200035F
S315080086B000221A70F7F7BAFD00F05EF970BD00BF28
S315080086C0AC09002008B540F65453C2F200031860FE
S315080086D040F65853C2F200031960FFF7F3FBFCE7B4
S315080086E02DE9F047002349F6D850C0F600004FF4AC
S315080086F0FA744AF2104113F80080C21892F801C0C1
S3150800870008EB0C0202FB044291FBF2F902FB191674
S3150800871036B94D4609F1FF3292B2B2F5806F03D3EE
S315080087200233242BE7D187E04746E2464FF4D0438D
S31508008730C4F2000300225A611A6842F400421A6021
S315080087401B6813F4004F09D04FF4D044C4F2000458
S31508008750FFF7B8FB236813F4004FF9D14FF4D04361
S31508008760C4F200031A6822F002021A601A6842F07C
S3150800877001021A605B6813F0010F09D14FF4D04467
S31508008780C4F20004FFF79EFB636813F0010FF9D0EB
S31508008790013F0AF1FF36360546EA0747013D3D43E4
S315080087A04FF4D043C4F20003DD611A6822F00102D7
S315080087B01A605B6813F0010F09D04FF4D044C4F275
S315080087C00004FFF77FFB636813F0010FF9D14FF43C
S315080087D0C843C4F20003D3F8002242F00102C3F8EA
S315080087E00022D3F81C2222F48042C3F81C22D3F8B4
S315080087F00C2242F48042C3F80C220022C3F8B022AD
S31508008800C3F8B422D3F8042222F48042C3F804221F
S31508008810D3F8142222F48042C3F81422D3F81C2277
S3150800882042F48042C3F81C22D3F8002222F0010247
S31508008830C3F80022BDE8F08749F6B450C0F6000038
S31508008840F021FFF73FFF71E738B504460D464FF4B0
S31508008850D043C4F200039B6813F0806F07D149F632
S31508008860B450C0F600004FF4A271FFF72BFF4FF487
S31508008870D043C4F20003D3F8802102F00102C3F802
S315080088808021D3F8802142F07C4242F40012C3F8DA
S315080088908021C3F88451E178A278120442EA016281
S315080088A021780A43617842EA0122C3F88821E179EE
S315080088B0A279120442EA016221790A43617942EAFD
S315080088C00122C3F88C21D3F8802142F00102C3F8B3
S315080088D080219B6813F0806F09D14FF4D044C4F20D
S315080088E00004FFF7EFFAA36813F0806FF9D038BDDC
S315080088F04FF4D043C4F20003DB6813F0030F39D0FA
S315080089004FF4D043C4F20003D3F8B02140F26763B2
S31508008910B3EB525F18BF002023D14FF4D043C4F203
S315080089200003D3F8B8210270D3F8B821120A4270AE
S31508008930D3F8B821120C8270D3F8B821120EC2707F
S31508008940D3F8BC210271D3F8BC21120A4271D3F8BC
S31508008950BC21120C8271D3F8BC311B0EC3710120E5
S31508008960FFE74FF4D043C4F20003DA6842F020026E
S31508008970DA6070470020704708B500F011FDA8B10D
S31508008980F7F708FC90B1FEF705FF00F02BFD00F0A5
S31508008990F3F920F0604020F07F024EF60853CEF23D
S315080089A000031A6000F0E8F94368984708BD00BF5D
S315080089B070B5561EB6B24AB14C1E0E44451A14F886
S315080089C0013F2B55FFF77EFAB442F8D170BD00BFC0
S315080089D0F8B507460024254649F62C66C0F6000673
S315080089E0FFF770FAA359BB420ED8311949680B44F0
S315080089F09F4209D249F62C63C0F6000305EB4502EF
S31508008A0003EB8203187AF8BD01350C346C2CE7D1D8
S31508008A10FF20F8BD2DE9F84380460068FFF7D8FF28
S31508008A20FF2830D0FBF704F8F320FBF721F8FBF713
S31508008A3025F801281CBF002408F1040904D1FBF716
S31508008A400DF80020BDE8F883D8F80060A71959F892
S31508008A500450FFF737FA38462946FBF78DF80828F9
S31508008A6007D1A359AB4206D10434B4F5007FEBD144
S31508008A7003E0002402E0002400E00124FAF7EEFFF8
S31508008A802046BDE8F8830020BDE8F88338B50446DB
S31508008A900D4640F65C53C2F20003984209D04FF4E3
S31508008AA04043C0F6000399420BD0FFF7B3FF20B945
S31508008AB017E040F66074C2F20004C5F3080393B9E0
S31508008AC003E040F65C54C2F2000423689D420CD0D1
S31508008AD0204640F8045B29464FF40072FFF768FF0A
S31508008AE003E0002038BD002038BD204638BD00BF51
S31508008AF02DE9F04106460C4617461D464FEA512811
S31508008B004FEA48280368B3F1FF3F06D140F8048BC3
S31508008B1041464FF40072FFF74BFF3368434505D0D3
S31508008B2030464146FFF7B2FF0646D0B13368E41A2D
S31508008B303444043408F50078FFF7C4F9331DE31A02
S31508008B40B3F5007F06D330464146FFF79FFF06463A
S31508008B5050B1041D17F8013B04F8013B013DEBD168
S31508008B6005E00020BDE8F0810020BDE8F081012085
S31508008B70BDE8F08140F66073C2F200034FF0FF32A1
S31508008B801A6040F65C53C2F200031A60704700BFD1
S31508008B9070B504460D461646FFF71AFFFF281BD088
S31508008BA0681E2044FFF714FFFF2817D0620A4FF407
S31508008BB04043C0F60003B3EB422F07BF40F65C50B4
S31508008BC0C2F2000040F66070C2F20000214632464A
S31508008BD02B46FFF78DFF70BD002070BD002070BDCD
S31508008BE0F8B505460E46FFF7F3FE0446701E284400
S31508008BF0FFF7EEFE0546FF2C18BFFF2833D0844248
S31508008C002BD8022C2BD90B282BD8FAF711FFF320D7
S31508008C10FAF72EFFFAF732FF01281EBF49F6FC566F
S31508008C20C0F60006022703D1FAF718FF0020F8BDA0
S31508008C30FFF748F936F814003946FAF765FF0828A9
S31508008C4003D0FAF70BFF0020F8BD0134E4B2A542C1
S31508008C50EED2FAF703FF0120F8BD0020F8BD002088
S31508008C60F8BD0020F8BD0020F8BD00BF00B583B0F0
S31508008C7040F65C53C2F200031B68B3F1FF3F08BF1E
S31508008C8001201CD040F65C53C2F2000399685A686A
S31508008C901144DA6811441A6911445A6911449A69E7
S31508008CA00A44D96953185B4202AA42F8043D4CF2B9
S31508008CB08810C0F600000421FFF76AFFFFE703B03B
S31508008CC05DF804FB4CF20402C0F600024FF4404380
S31508008CD0C0F6000310681B6818444CF20803C0F677
S31508008CE000031B6818444CF20C03C0F600031B680B
S31508008CF018444CF21003C0F600031B6818444CF2E3
S31508008D001403C0F600031B6818444CF21803C0F697
S31508008D1000031B6818444CF28813C0F600031B684E
S31508008D201844D0F1010038BF0020704708B540F656
S31508008D305C53C2F200031B68B3F1FF3F06D040F64E
S31508008D405C50C2F20000FFF765FE88B140F660731A
S31508008D50C2F200031B68B3F1FF3F0BD040F6607008
S31508008D60C2F20000FFF756FE003018BF012008BD0A
S31508008D70002008BD012008BD4FF44040C0F60000A1
S31508008D80704700BF38B504464FF4A050C4F201003E
S31508008D908021FBF779F990B14FF4A050C4F2010095
S31508008DA02146FBF769F94FF4A054C4F20104802563
S31508008DB020462946FBF768F90028F9D001E000208B
S31508008DC038BD012038BD00BF10B504464FF4A05089
S31508008DD0C4F201002021FBF757F9012808D14FF406
S31508008DE0A050C4F20100FBF74BF92070012010BD1A
S31508008DF0002010BD10B584B04FF4614300930023E2
S31508008E00ADF80430ADF80630ADF80830ADF80C30E2
S31508008E100C23ADF80A304FF4A054C4F201042046DE
S31508008E206946FBF7ABF820460121FBF717F904B0B2
S31508008E3010BD00BF2DE9F04106460C46402906D96B
S31508008E4049F69860C0F600007721FFF73BFC2046FC
S31508008E50FFF798FF012806D049F69860C0F600008B
S31508008E607B21FFF72FFC2546ACB1002449F698670D
S31508008E70C0F600074FF08408FFF724F8305DFFF7C7
S31508008E8081FF012803D038464146FFF71BFC013411
S31508008E90A3B2AB42F0D3BDE8F08100BF10B50446DB
S31508008EA041F2A913C2F200031B78D3B941F2641048
S31508008EB0C2F20000FFF788FF012838D141F2641397
S31508008EC0C2F200031B78A3B341F2A913C2F200034E
S31508008ED001221A7041F2A813C2F20003002018708A
S31508008EE010BD41F2A813C2F200031878144B1844B7
S31508008EF0FFF76AFF01281ED141F2A813C2F2000348
S31508008F001A780132D2B21A7041F26413C2F200031F
S31508008F101B78934211D120460949FFF749FD41F2D2
S31508008F20A913C2F2000300221A70012010BD002006
S31508008F3010BD002010BD002010BD002010BD00BFD0
S31508008F406511002038B504460D46012807D949F6AB
S31508008F50BC60C0F6000040F29F11FFF7B3FB41F278
S31508008F60F013C2F2000304EB440203EBC2035A7C7B
S31508008F701B7C9A4220D041F2F013C2F2000304EBA4
S31508008F80440203EBC203DA681570597C013159743F
S31508008F90DA680132DA605B689A420FD941F2F01357
S31508008FA0C2F200036200111953F83110144403EB9E
S31508008FB0C403D960012038BD002038BD012038BD62
S31508008FC038B504460D46012807D949F6BC60C0F6EF
S31508008FD0000040F2C111FFF775FB41F2F013C2F22F
S31508008FE0000304EB440203EBC2035B7CFBB141F2D2
S31508008FF0F013C2F2000303EBC2039A6812782A70D0
S31508009000597C013959749A6801329A605B689A42A8
S315080090100FD941F2F013C2F200036200111953F896
S315080090203110144403EBC4039960012038BD0020B5
S3150800903038BD012038BD00BF10B582B041F2F0132B
S31508009040C2F200030020987403F118025A61012144
S3150800905083F82A10D86241F2EC11C2F200010A60C4
S315080090604021197441F2A821C2F200014C1C9C60EF
S31508009070DC6058741C6001F140045C600870002ACA
S315080090803DD041F2EC11C2F20001D86A08604021D5
S3150800909083F8281041F22021C2F20001481C186208
S315080090A05862002483F82940986101F1400353600F
S315080090B0927C0A7041F2A823C2F200031B78FF2BA8
S315080090C001D0FF2A06D149F6BC60C0F600007E2111
S315080090D0FFF7F8FA40F28003C2F20003009341F268
S315080090E0F020C2F20000012140F24C02C2F2000256
S315080090F040F22003C2F20003F7F7F2FB06E041F262
S315080091002023C2F20003FF221A70DCE702B010BD6A
S3150800911008B541F2F020C2F20000F8F771FC002011
S31508009120F7F732F808BD00BF2DE9F84307460C46A5
S315080091303F2906D949F6BC60C0F600009F21FFF713
S31508009140C1FA41F2A823C2F2000318782146FFF7B4
S31508009150F9FE012806D049F6BC60C0F60000A32136
S31508009160FFF7B0FA2646D4B1002441F2A825C2F288
S31508009170000549F6BC68C0F600084FF0AC09FEF7D2
S31508009180A1FE2878395DFFF7DDFE012803D04046A9
S315080091904946FFF797FA0134A3B2B342EFD3BDE8C5
S315080091A0F88300BF10B5044641F2F020C2F2000071
S315080091B0F8F730FC41F2EC23C2F200031B7803BB3C
S315080091C041F22023C2F20003187841F2AC11C2F230
S315080091D00001FFF7F5FE01283ED141F2AC13C2F2B9
S315080091E000031B78002B39D041F2EC23C2F20003AE
S315080091F001221A7041F2A423C2F20003002018705B
S3150800920010BD41F22023C2F2000341F2A422C2F2A9
S31508009210000211781878144B1944FFF7D1FE01287B
S315080092201ED141F2A423C2F200031A780132D2B247
S315080092301A7041F2AC13C2F200031B78934211D1A3
S3150800924020460949FFF7B4FB41F2EC23C2F20003BA
S3150800925000221A70012010BD002010BD002010BD8C
S31508009260002010BD002010BDAD1100202DE9F043EF
S3150800927083B041F2A823C2F200031C78012C07D957
S3150800928049F6BC60C0F6000040F2E111FFF71AFA91
S3150800929041F2F013C2F2000304EB440403EBC403E7
S315080092A05B7CBBB3402B34BF99464FF04009B9F1FC
S315080092B0000F23D041F26422C2F20002541E09F1C3
S315080092C0FF3652FA86F641F2A825C2F2000549F69B
S315080092D0BC67C0F6000740F2291828780DF1070187
S315080092E0FFF76EFE012803D038464146FFF7EAF934
S315080092F09DF8072004F8012FB442EED141F2F02080
S31508009300C2F20000812141F26422C2F200024B46F9
S31508009310F8F714FB03B0BDE8F08300BF2DE9F84366
S3150800932041F2F023C2F2000300EB800003EBC00316
S31508009330B3F88C73DFB1002441F22026C2F200068E
S3150800934049F6BC68C0F600084FF4A4793578F7F7F3
S31508009350B3F8015D2846FFF7F5FD012803D040461E
S315080093604946FFF7AFF90134A3B29F42EED8F7F7A3
S31508009370A3F8024641F2F020C2F200000121402380
S31508009380F8F7C0FABDE8F88308B5FFF7F3FB08BDA0
S3150800939008B5FFF7FDFB08BD08B5FFF721FC08BDBA
S315080093A008B5FFF78FFC08BD08B5FFF75FFC10B1DD
S315080093B0FFF7BCFC08BD002008BD00BF4EF2100335
S315080093C0CEF2000300221A6049F23F01C0F2020100
S315080093D059609A600521196041F6E403C2F2000358
S315080093E01A6070474EF21003CEF2000300221A608C
S315080093F0704700BF4EF21003CEF200031B6813F449
S31508009400803F1FBF41F6E403C2F200031A68013227
S3150800941018BF1A60704700BF08B5FFF7EBFF41F6A3
S31508009420E403C2F20003186808BD00BF08B549F690
S31508009430E060C0F600003621FFF744F908BD00BF1A
S3150800944010B572B640F20002C2F2000240F2EC0316
S31508009450C2F200039A4210D2131D0E4CE41A24F0ED
S3150800946003040434002310464AF21001C0F6000132
S315080094705A581A500433A342FAD1074807494FF0FD
S3150800948000028842B8BF40F8042BFADBF6F730FF33
S3150800949010BD00BFEF00002000010020642E002050
S315080094A00F2AF0B445D940EA01039B0745D1A2F13A
S315080094B010070C4603463F0900EB071610362568C9
S315080094C01033103443F8105C54F80C5C43F80C5C09
S315080094D054F8085C43F8085C54F8045C43F8045CE8
S315080094E0B342ECD17B1C02F00F0CBCF1030F4FEA20
S315080094F003131944034422D90E461D46644656F8FA
S31508009500047B043C032C45F8047BF8D8ACF104042E
S3150800951002F0030224F0030404342344214432B144
S315080095200A4411F8014B914203F8014BF9D1F0BCFA
S3150800953070470346002AF3D1F9E70346F0E7624687
S31508009540002AEDD1F3E700BF8307F0B448D0541ED4
S31508009550002A43D0CDB2034602E0002C3ED0144682
S3150800956003F8015B13F0030F04F1FF32F5D1032C66
S315080095702DD9CDB20F2C45EA052545EA054518D95A
S31508009580A4F1100703F110061A463F0906EB071661
S315080095901560103242F80C5C42F8085C42F8045C2C
S315080095A0B242F5D104F00F040137032C03EB07137D
S315080095B00DD91E462246043A46F8045B032AFAD811
S315080095C0221F04F0030422F00302043213442CB1D0
S315080095D0C9B21C4403F8011BA342FBD1F0BC704777
S315080095E014460346C3E700BF2F64656D6F70726F3C
S315080095F0675F6F6C696D65785F73746D3332653458
S3150800960030372E73726563002F626F6F746C6F67E5
S315080096102E7478740000000057696E555342204234
S31508009620756C6B2044657669636500004F70656EDE
S31508009630424C5420557365720000000030303030BB
S315080096403030303030353043000000004465666104
S31508009650756C740057696E5553422042756C6B20C1
S31508009660496E746572666163650000002E2F6C6929
S31508009670622F7569702F6E65746465762E630000B7
S31508009680222A3A3C3E3F7C7F000000002B2C3B3DC3
S315080096905B5D0000809A90418E418F804545454923
S315080096A049498E8F9092924F994F555559999A9B41
S315080096B09C9D9E9F41494F55A5A5A6A7A8A9AAABBB
S315080096C0AC21AEAFB0B1B2B3B4B5B6B7B8B9BABBE0
S315080096D0BCBDBEBFC0C1C2C3C4C5C6C7C8C9CACB44
S315080096E0CCCDCECFD0D1D2D3D4D5D6D7D8D9DADB34
S315080096F0DCDDDEDFE0E1E2E3E4E5E6E7E8E9EAEB24
S31508009700ECEDEEEFF0F1F2F3F4F5F6F7F8F9FAFB13
S31508009710FCFDFEFF01030507090E10121416181C9E
S315080097201E000000610062006300640065006600B8
S315080097306700680069006A006B006C006D006E00C7
S315080097406F00700071007200730074007500760077
S315080097507700780079007A00A100A200A300A5008E
S31508009760AC00AF00E000E100E200E300E400E50041
S31508009770E600E700E800E900EA00EB00EC00ED008F
S31508009780EE00EF00F000F100F200F300F400F5003F
S31508009790F600F800F900FA00FB00FC00FD00FE00E8
S315080097A0FF00010103010501070109010B010D0174
S315080097B00F01110113011501170119011B011D01E3
S315080097C01F01210123012501270129012B012D0153
S315080097D02F0131013301350137013A013C013E01C0
S315080097E0400142014401460148014B014D014F0128
S315080097F0510153015501570159015B015D015F0193
S31508009800610163016501670169016B016D016F0102
S3150800981071017301750177017A017C017E0192015C
S31508009820B103B203B303B403B503B603B703B8036E
S31508009830B903BA03BB03BC03BD03BE03BF03C0031E
S31508009840C103C303C403C503C603C703C803C903C7
S31508009850CA033004310432043304340435043604AC
S315080098603704380439043A043B043C043D043E04F6
S315080098703F044004410442044304440445044604A6
S315080098804704480449044A044B044C044D044E0456
S315080098904F045104520453045404550456045704FF
S315080098A0580459045A045B045C045E045F0470217E
S315080098B071217221732174217521762177217821EE
S315080098C079217A217B217C217D217E217F2141FFFF
S315080098D042FF43FF44FF45FF46FF47FF48FF49FF56
S315080098E04AFF4BFF4CFF4DFF4EFF4FFF50FF51FF06
S315080098F052FF53FF54FF55FF56FF57FF58FF59FFB6
S315080099005AFF0000C700FC00E900E200E400E0009E
S31508009910E500E700EA00EB00E800EF00EE00EC00E7
S31508009920C400C500C900E600C600F400F600F2004F
S31508009930FB00F900FF00D600DC00A200A300A5008A
S31508009940A7209201E100ED00F300FA00F100D10032
S31508009950AA00BA00BF001023AC00BD00BC00A100DD
S31508009960AB00BB0091259225932502252425612568
S315080099706225562555256325512557255D255C25E0
S315080099805B251025142534252C251C2500253C256A
S315080099905E255F255A2554256925662560255025A7
S315080099A06C2567256825642565255925582552257A
S315080099B053256B256A2518250C25882584258C258D
S315080099C090258025B103DF009303C003A303C303D7
S315080099D0B500C403A6039803A903B4031E22C6034D
S315080099E0B50329226122B10065226422202321239E
S315080099F0F7004822B0001922B7001A227F20B200C9
S31508009A00A025A0004100420043004400450046004E
S31508009A104700480049004A004B004C004D004E00E4
S31508009A204F00500051005200530054005500560094
S31508009A305700580059005A002100E0FFE1FFE5FFF2
S31508009A40E2FFE3FFC000C100C200C300C400C500B6
S31508009A50C600C700C800C900CA00CB00CC00CD00AC
S31508009A60CE00CF00D000D100D200D300D400D5005C
S31508009A70D600D800D900DA00DB00DC00DD00DE0005
S31508009A807801000102010401060108010A010C011E
S31508009A900E01100112011401160118011A011C0108
S31508009AA01E01200122012401260128012A012C0178
S31508009AB02E01300132013401360139013B013D01E5
S31508009AC03F0141014301450147014A014C014E014D
S31508009AD0500152015401560158015A015C015E01B8
S31508009AE0600162016401660168016A016C016E0128
S31508009AF0700172017401760179017B017D01910182
S31508009B00910392039303940395039603970398038B
S31508009B1099039A039B039C039D039E039F03A0033B
S31508009B20A103A303A403A503A603A703A803A903E4
S31508009B30AA031004110412041304140415041604C9
S31508009B401704180419041A041B041C041D041E0413
S31508009B501F042004210422042304240425042604C3
S31508009B602704280429042A042B042C042D042E0473
S31508009B702F0401040204030404040504060407046C
S31508009B80080409040A040B040C040E040F046021DB
S31508009B90612162216321642165216621672168218B
S31508009BA069216A216B216C216D216E216F2121FFAC
S31508009BB022FF23FF24FF25FF26FF27FF28FF29FF73
S31508009BC02AFF2BFF2CFF2DFF2EFF2FFF30FF31FF23
S31508009BD032FF33FF34FF35FF36FF37FF38FF39FFD3
S31508009BE03AFF0000FFFFFFFFFFFF00004F70656EA2
S31508009BF0424C54002E2E2F2E2E2F2E2E2F536F759D
S31508009C007263652F66696C652E6300004669726D1E
S31508009C107761726520757064617465207265717507
S31508009C206573742064657465637465640A0D000061
S31508009C304F70656E696E67206669726D77617265C9
S31508009C402066696C6520666F722072656164696E4C
S31508009C50672E2E2E000000004552524F520A0D0064
S31508009C604F4B0A0D000000005374617274696E67E9
S31508009C70207468652070726F6772616D6D696E67B2
S31508009C802073657175656E63650A0D0050617273A0
S31508009C90696E67206669726D776172652066696CA0
S31508009CA06520746F206F627461696E2065726173D6
S31508009CB0652073697A652E2E2E0000004572617341
S31508009CC0696E67200000000020627974657320665B
S31508009CD0726F6D206D656D6F7279206174203078B2
S31508009CE00000000052656164696E67206C696E65E4
S31508009CF02066726F6D2066696C652E2E2E4552524F
S31508009D004F520A0D00000000496E76616C696420A6
S31508009D10636865636B73756D20666F756E642E2E4A
S31508009D202E4552524F520A0D0000000050726F67BE
S31508009D3072616D6D696E672000000000206279749B
S31508009D40657320746F206D656D6F7279206174205C
S31508009D503078000057726974696E672070726F6791
S31508009D6072616D20636865636B73756D2E2E2E00A8
S31508009D70436C6F73696E67206669726D7761726589
S31508009D802066696C650A0D004669726D77617265B1
S31508009D902075706461746520737563636573736693
S31508009DA0756C6C7920636F6D706C657465640A0DEB
S31508009DB0000000002E2E2F2E2E2F2E2E2F536F75BD
S31508009DC07263652F41524D434D345F53544D3332C0
S31508009DD02F63616E2E630000050206020603070361
S31508009DE00803090309040A040B040C040C050D05F1
S31508009DF00E050F050F0610061007100800000800CC
S31508009E0010001800200028003000380040004800E4
S31508009E10500058008000880090009800A000A80014
S31508009E20B000B800C000C800D000D80000C00008C4
S31508009E3000400000030000000000010800000100C7
S31508009E4004000000000002080000020005000000EF
S31508009E5000000408000002000600000000000608D2
S31508009E6000000200070000000000080800000200C9
S31508009E700800000000000A080000020009000000AF
S31508009E8000000C08000002000A00000000000E088E
S31508009E90000002000B0000002E2E2F2E2E2F2E2E35
S31508009EA02F536F757263652F41524D434D345F537F
S31508009EB0544D33322F756172742E63002E2E2F2E59
S31508009EC02E2F2E2E2F536F757263652F41524D43D9
S31508009ED04D345F53544D33322F7573622E63000031
S31508009EE02E2E2F2E2E2F2E2E2F536F757263652F23
S31508009EF041524D434D345F53544D33322F474343FC
S31508009F002F766563746F72732E630000002020201D
S31508009F10202020202020282828282820202020200B
S31508009F2020202020202020202020202020881010DB
S31508009F301010101010101010101010101004040437
S31508009F4004040404040404101010101010104141F5
S31508009F5041414141010101010101010101010101E3
S31508009F6001010101010101011010101010104242F7
S31508009F7042424242020202020202020202020202B3
S31508009F800202020202020202101010102000000053
S31508009F9000000000000000000000000000000000B3
S31508009FA000000000000000000000000000000000A3
S31508009FB00000000000000000000000000000000093
S31508009FC00000000000000000000000000000000083
S31508009FD00000000000000000000000000000000073
S31508009FE00000000000000000000000000000000063
S31508009FF00000000000000000000000000000000053
S3150800A0000000000000000000000000000000000042
S3150800A01009022000010100C0320904000002FF0005
S3150800A0200000070581024000FF070501024000FF06
S3150800A03089040008710400080904000800000000EB
S3150800A04000000000F1030008FD030008DD03000816
S3150800A0500000000000000000CD030008C504000849
S3150800A060D504000805050008E504000825050008CC
S3150800A07045050008650500080403090412011001D6
S3150800A0800000004045012300000101020301000011
S3150800A09085050008890500088D0500089105000852
S3150800A0A099050008A1050008AD050008A0000020D4
S3150800A0B069080008B107000861070008C906000812
S3150800A0C031070008AD06000895060008D9060008FD
S3150800A0D0E9060008F9060008110700080100000053
S3150800A0E0010000000000000001020304010203044D
S3110800A0F006070809040000000C9F000881
S70508000000F2
